:046F4E0001000145F8
:1069C000AF50055074D02FF582E4341DF583E5995E
:1069D000F022D3E5309400E52F94002290000FE0E0
:0369E0006403222B
:0300030002577130
:0B577100C0E0C083C082C0D075D0082B
:10577C00852E82852D83E493FF201404C4540FFFDF
:10578C00430FF08F80C284D28500C2870000D2877D
:10579C00007580FF7580FEC284C28500C287000040
:1057AC00D287007580FF30140CC214052EE52E70C4
:0957BC0006052D8002D214D2A8CA
:0957C500D0D0D082D083D0E032B4
:03000B0002195F78
:10195F00C0E0C0F0C083C082C0D075D008758CD8ED
:10196F00758A92D28C12421412630EE531D3940011
:10197F0040171531E53164056009E531640F6003E7
:10198F00021B71126C05021B71753114E54ED39455
:10199F00004002154EE54FD394004002154FE53A33
:1019AF00D394004002153AE54BD394004002154BF7
:1019BF00154CE54C123A4A1B63001B38011B1002F1
:1019CF001AE8031A65041A4C051A33061A1A071A6D
:1019DF00010819E80900001B6ED3E52C9400E52BD4
:1019EF0094005003021B71E52C152C704D152B0222
:1019FF001B71D3E5379400E53694005003021B7139
:101A0F00E537153770021536021B71D3E548940080
:101A1F00E54794005003021B71E548154870021505
:101A2F0047021B71D3E54A9400E549940050030225
:101A3F001B71E54A154A70021549021B71D3E52A3D
:101A4F009400E52994005003021B71E52A152A70B2
:101A5F00021529021B717885E6FF7003021B71EFD7
:101A6F00B40105900524801BEFB402101269D24017
:101A7F002FE53015307002152F021B71EFB4030CD8
:101A8F00900526E0F52FA3E0F5308028EFB404127F
:101A9F001269D2400BE53015307002152F021B7101
:101AAF008012EF64057003021B71EFB4060C752FE3
:101ABF0002753058788506021B71EF6407600302C8
:101ACF001B711269D2400BE53015307002152F02D1
:101ADF001B7178857600021B71D3E5399400E538C8
:101AEF0094004008E539153970021538D3E53C9458
:101AFF0000E53B9400406BE53C153C7002153B80C4
:101B0F0061D3E5579400E55694004008E557155703
:101B1F0070021556D3E5559400E55494004043E503
:101B2F00551555700215548039D3E5359400E534B9
:101B3F0094004008E535153570021534301523D360
:101B4F00E5339400E53294004018E53315337012F5
:101B5F001532800EE551D394004004155180007565
:0D1B6F004C0AD0D0D082D083D0F0D0E0322C
:03001300023EDFCB
:0D3EDF00C0E0C0F0C083C082C0D075D0101C
:103EEC00E545C394504003023FA3202403023FA3A3
:103EFC00300C03023FA3E5A0540FF5587D077F015A
:103F0C00124ED95067202364E545700DE558B40C6A
:103F1C0008201105D211023FA320034A2011471299
:103F2C003FAE50047F0180027F0F126ED190000FC4
:103F3C00E0FF64016012EFB40302800C90000FE00C
:103F4C00B40209123FAE50047F80801290000FE043
:103F5C00B4020E7D037F07124ED940057FA01200DC
:103F6C0016754202D20390053CE0F53A7D087F05B8
:103F7C00124ED9502290002BE0B55807202304D2C2
:103F8C00268014053EE53EAE3D7002053D14F582DB
:073F9C008E83E558F0054596
:103FA300D0D0D082D083D0F0D0E0327D037F07120F
:033FB3004ED922C2
:030023000263E78E
:1063E700C0E0C083C082C0D075D018309819C29859
:1063F700E599B40A081269C0755000800AE550C3D0
:10640700949050031269C0309902C299D0D0D082BB
:05641700D083D0E0324B
:03003B0002492057
:0D492000C0E0C0F0C083C082C0D075D018C8
:10492D00C2CEE546C3941040030249B830257C2021
:10493D000C79AFA07804EF08800123D8FDF5595309
:10494D00590F7D077F02124ED95035202332E5468F
:10495D00700CE559B40C07201304D213804D2004BC
:10496D001920131690000FE0B4020F7F0A126ED1BA
:10497D007F80120016754202D20490053CE0F53A94
:10498D007D087F05124ED9502290002BE0B55907B6
:10499D00202304D22880140540E540AE3F70020567
:0B49AD003F14F5828E83E559F00546AB
:0B49B800D0D0D082D083D0F0D0E0320D
:104B8500E4F55AF55B755C1E755DFF855B82855A9C
:104B950083E0F55E635EFFE55EF0E0655E6003124F
:104BA5006F52635EFF855B82855A83E55EF0E06543
:104BB5005E6003126F52055BE55B7002055AE55DA9
:104BC500155D7002155CD3E55D9400E55C940050BD
:104BD500BA75985A758921758845758DE7758780E9
:104BE500758CD8758AEF75C90275C808753D1E752F
:104BF5003E60753F1E7540B075B701D2A9D2E8D2A7
:0F4C0500AA75C64C75EEFF75FEFFD2AF1266E2C0
:014C1400227D
:026F520080FEBF
:10699D00202F0F90053AE0F54EE54ED394004012AE
:1069AD0080F7302F0D90053AE0F54FE54FD3940069
:0369BD0050F9226C
:1069550030310AD215900024E04420800DC2157F05
:1069650008126F12900024E054DFF0FD7F247E00B2
:046975001263B122D6
:102EB6008F70E570640170292030047F01805620F0
:102EC6003003022FB1122FC24003022FB1122FCAB4
:102ED600500C122FB2301503022FB1022FA7022F6A
:102EE60067E570640270202030047F02802720305E
:102EF60003022FB1122FD24003022FB11269DC70E8
:102F060003022FB1022F81E57064036003022FB123
:102F16002030057F03026F12303024122FC2501F5B
:102F2600122FD2501A1269DC6015122FCA500B7F6D
:102F36000B122FDA201574022FA77F03022FAE3053
:102F46003023122FE8501E7D017F02124ED9401504
:102F56007D017F07124ED95008122FB220154C80E2
:102F6600407F018043303017122FE840127D017FE9
:102F760002124ED950091269DC60047F02802930A2
:102F860030297D017F01124ED950201269DC701B59
:102F96007D017F07124ED9500D7F09122FDA2015B9
:102FA6000AD2310269557F01126F25227F09126FFD
:102FB60025900536E0F532A3E0F533227D017F0149
:102FC600124ED9227D017F07124ED9227D017F0242
:102FD600124ED922126F25900536E0F532A3E0F5A0
:0A2FE60033227D017F01124ED92233
:104C1500C2957FFF126F12124B857F0712634550B5
:104C25000512003E80031260CCD28C7F08126345CA
:104C350050051242D480FEC22B12689B9000D1E031
:104C4500FF7C117D00125C06125D7990000FE0B4C7
:104C5500010512281D801090000FE0FF640260041A
:104C6500EFB40303123251123D1E301E11E542709E
:104C75000DE52754A060077FA0126ED1C21E7D07E7
:104C85007F05124ED94002C200E552C3940A50BBBB
:104C95003015B8E533453270B2C23112695580AB73
:104A5C00EF253EFFEE353DCF2401FDE43FFC22AFB8
:104A6C005A7E00EF2403FDEE33FC22E53E255AF579
:104A7C0082E4353DF58322E540255AF582E4353F45
:104A8C00F58322E56F256DF582E4356EF583E0FF45
:104A9C00E56F256DF582E4356EF58322E55A240227
:104AAC00FFE433FE22E56C2401FFE433FEC3E56D25
:104ABC009FEE6480F874809822EF2540FFEE353F1E
:104ACC0022C2017FF47E01126C5BE56C25E0F56C73
:104ADC00756D0122E55C2EF582E4355BF583E0FD16
:084AEC0022753D1E753E60229B
:106C5B00EF1FAA0670011ED39400EA9400400BE4C8
:0A6C6B00FDEDC394C850E90D80F759
:016C750022FC
:105170008F5BE55BB401197D017F06124ED9500C9F
:105180009000B1E0FF7C0D7D00125C067885062260
:10519000E55BB402131251E250439000B2E0FF7C91
:1051A0000D7D20125C068035E55BB404161251E2D9
:1051B000500C9000B4E0FF7C0D7D60125C06788599
:1051C000760622E55BB403197D027F06124ED950A4
:1051D0000C9000B3E0FF7C0D7D40125C0678857674
:0A51E00001227D027F06124ED92243
:104ED900BF0107900020E0FE8048BF020790002133
:104EE900E0FE803EBF0307900022E0FE8034BF044D
:104EF90007900023E0FE802ABF0507900024E0FE0A
:104F09008020BF0607900025E0FE8016BF070790A6
:104F19000026E0FE800CBF0807900027E0FE800213
:104F2900E4FEBD0103EE1322BD0204EEA2E122BD9F
:104F39000304EEA2E222BD0404EEA2E322BD0504AD
:104F4900EEA2E422BD0604EEA2E522BD0704EEA20C
:074F5900E622BD0802EE3361
:014F6000222E
:101D7D00124AED900100E0F55A124A77E0123A4A04
:101D8D001DAC011DE1021E16031E4B041E80051E17
:101D9D00B5061EEA071F1A081F460900001F70121C
:101DAD004A77A3E0B40A15E55A124AAAE545B507E4
:101DBD000BE4B506077D017F01021F2E124A6BE56C
:101DCD00456D7001EC6003021F70124A5CC2297FE1
:101DDD0001021F43124A77A3E0B40A15E55A124ACD
:101DED00AAE545B5070BE4B506077D017F02021F85
:101DFD002E124A6BE5456D7001EC6003021F7012E7
:101E0D004A5CC2297F02021F43124A77A3E0B40A3B
:101E1D0015E55A124AAAE545B5070BE4B506077D47
:101E2D00017F03021F2E124A6BE5456D7001EC60B8
:101E3D0003021F70124A5CC2297F03021F43124A1C
:101E4D0077A3E0B40A15E55A124AAAE545B5070B82
:101E5D00E4B506077D017F04021F2E124A6BE5458E
:101E6D006D7001EC6003021F70124A5CC2297F0481
:101E7D00021F43124A77A3E0B40A15E55A124AAA83
:101E8D00E545B5070BE4B506077D017F05021F2E5D
:101E9D00124A6BE5456D7001EC6003021F70124A2A
:101EAD005CC2297F05021F43124A77A3E0B40A15CD
:101EBD00E55A124AAAE545B5070BE4B506077D01BB
:101ECD007F06021F2E124A6BE5456D7001EC600313
:101EDD00021F70124A5CC2297F06021F43124A7705
:101EED00A3E0B40A14E55A124AAAE545B5070AE477
:101EFD00B506067D017F078028124A6BE5456D709A
:101F0D0001EC705F124A5CC2297F078029124A7763
:101F1D00A3E0B40A0F124A77A3A3E070077D017FF7
:101F2D0008024E4E124A6BE5456D7001EC7034128D
:101F3D004A5CC2297F08020FF1124A77A3A3E07011
:101F4D0022124A77A3E024F96008147016E4FF0208
:101F5D005F567FF47E01126C5B7D5E7F021266B868
:031F6D001242D449
:011F7000224E
:101B7C00753F1E7540B0900108E0F55A124A83E09B
:101B8C00123A4A1BAE011BE6021C1E031C56041C17
:101B9C008E051CC6061CFE071D31081D66090000BB
:101BAC001D7C124A83A3E0B40A13124AA8E546B579
:101BBC00070BE4B506077D017F01021D49AF5A12E0
:101BCC004A6DE5466D7001EC6003021D7C124AC53E
:101BDC00124A63D2297F01021D63124A83A3E0B427
:101BEC000A13124AA8E546B5070BE4B506077D01B2
:101BFC007F02021D49AF5A124A6DE5466D7001EC29
:101C0C006003021D7C124AC5124A63D2297F02026C
:101C1C001D63124A83A3E0B40A13124AA8E546B521
:101C2C00070BE4B506077D017F03021D49AF5A126D
:101C3C004A6DE5466D7001EC6003021D7C124AC5CD
:101C4C00124A63D2297F03021D63124A83A3E0B4B4
:101C5C000A13124AA8E546B5070BE4B506077D0141
:101C6C007F04021D49AF5A124A6DE5466D7001ECB6
:101C7C006003021D7C124AC5124A63D2297F0402FA
:101C8C001D63124A83A3E0B40A13124AA8E546B5B1
:101C9C00070BE4B506077D017F05021D49AF5A12FB
:101CAC004A6DE5466D7001EC6003021D7C124AC55D
:101CBC00124A63D2297F05021D63124A83A3E0B442
:101CCC000A13124AA8E546B5070BE4B506077D01D1
:101CDC007F06021D49AF5A124A6DE5466D7001EC44
:101CEC006003021D7C124AC5124A63D2297F060288
:101CFC001D63124A83A3E0B40A12124AA8E546B542
:101D0C00070AE4B506067D017F078031AF5A124AF7
:101D1C006DE5466D7001EC7057124AC5124A63D2DC
:101D2C00297F078032124A83A3E0B40A13124AA80F
:101D3C00E546B5070BE4B506077D017F08024E4E5C
:101D4C00AF5A124A6DE5466D7001EC7023124AC50C
:101D5C00124A63D2297F08020FF1124A83A3A3E02F
:101D6C00700E124A83A3E024F870057F01125F56AF
:011D7C002244
:0447D3008C5B8D5C12
:1047D700055CE55C7002055B14F5828C83E0F9707B
:1047E7000302487AEF7005124AED8009BF0106758A
:1047F7003F1E7540B0302946EF7007E965456002F6
:10480700C322BF0107E965466002C322E4FEEEC387
:10481700995029EF700F124AE0E53E2E124A7BE0CD
:104827006D6002C322EF6401700F124AE0E5402E6B
:10483700124A87E06D6002C3220E80D2D32220295C
:1048470033E4FEEEC3995029EF700F124AE0E53EBC
:104857002E124A7BE06D6016C322EF6401700F12BF
:104867004AE0E5402E124A87E06D6002C3220E80BF
:04487700D2D322C3B3
:01487B00221A
:060FF1008F5BAB05AA04B2
:100FF7007D027F07124ED95011E55BB4050C8B8239
:101007008A83E06405700302125E7D017F07124E3A
:10101700D95011E55BB4050C8B828A83E0640670B6
:101027000302125EC22AEB24FFF582EA34FFF5833E
:10103700E0F55D8B828A83E0FFF55EA3E0F9F55F5B
:10104700EF123A4A106701106E02107503107C0404
:10105700108305108A061091071098080000109D4C
:10106700755C01D22A802F755C02D22A8028755CB4
:1010770004D22A8021755C08D22A801A755C10D2A6
:101087002A8013755C20D22A800C755C40D22A8096
:1010970005755C80D22AE924FE700302115F24F8EB
:1010A700605C24096003021171E55BB401059000DF
:1010B700208045E55BB40205900021803BE55BB4E9
:1010C70003059000228031E55BB40405900023807E
:1010D70027E55BB40505900024801DE55BB4060594
:1010E7009000258013E55BB407059000268009E58D
:1010F7005B64087077900027E0455CF0806EE55BE5
:10110700B401059000208045E55BB40205900021FD
:10111700803BE55BB403059000228031E55BB404B6
:10112700059000238027E55BB40505900024801D0A
:10113700E55BB406059000258013E55BB4070590D1
:1011470000268009E55B64087022900027E0FFE530
:101157005CF4FEEF5EF08014E55BB4050D8B828ACC
:1011670083E0FFD22F12297EC22AC22A202A030235
:10117700125EE55BB40109900020E0FD7F208060EE
:10118700E55BB40209900021E0FD7F218052E55B19
:10119700B40309900022E0FD7F228044E55BB4049C
:1011A70009900023E0FD7F238036E55BB4050990B5
:1011B7000024E0FD7F248028E55BB4060990002524
:1011C700E0FD7F25801AE55BB40709900026E0FD66
:1011D7007F26800CE55BB4080C900027E0FD7F2795
:1011E7007E001263B1126D70D2AF2029047F018097
:1011F700027F02126F25A229922F12699DAD5DE42D
:10120700FF1266B8AD5EE4FF1266B8E55FB401048D
:101217007D388007E55FB40A077D367F061266B81A
:10122700E55BB405031265157D077F05124ED9509E
:101237000A200007C2307F03122EB67D017F0112FC
:101247004ED94005C230122EB67D017F02124ED90B
:071257004005C230122EB663
:01125E00226D
:024E4E008F5B78
:104E5000ED24FF922F12699DE55B123A4A4E7901CB
:104E60004E7E024E83034E88044E8D054E92064EB2
:104E700097074E9C0800004EA290002080219000D1
:104E800021801C9000228017900023801290002423
:104E9000800D90002580089000268003900027E078
:104EA000F55CE55C6024755E01E4F55DE55C30E091
:104EB00007AD5EE4FF1266B8E55CC313F55C055E02
:104EC000055DE55DC3940840E3227D187F0212660C
:084ED000B87D537F021266B8A1
:014ED80022B7
:10634500C2AFD284C285BF070BC28600E580A2E238
:10635500922A8019BF080BC28600E580A2E3922A23
:10636500800BBF0508C28600E58013922AD286D22B
:0563750085D2AFA22A51
:01637A002200
:1045BE00C229D22DE4FF1259E77D2E7F031266B871
:1045CE007D607F021266B87F03126F123024FD20C9
:1045DE0024FDE5456407703B7E017F50124AED8F46
:1045EE00828E837407F07D01E53E2D124A7BE582B3
:1045FE0024FFF582E58334FFF583E0F9EF2DF58294
:10460E00E43EF583E9F00DBD08DED2297F647E001D
:10461E00126C5B7F081263455043302995D22DE40E
:10462E00FF1259E77D607F021266B87D327F061257
:10463E0066B87D1E7F051266B8C22DE4FF1259E7DB
:10464E007C017D507B087F507E011255E97F081258
:10465E00634550097F327E00126C5B80F07F647E72
:04466E0000126C5B6F
:014672002225
:025580008F5A40
:10558200900138E0F55BE55A7020E55B124AAAE526
:10559200456F7001EE704F7460255BF582E4341E36
:1055A200AF82F55D8F5E7F408024E55A64017036DC
:1055B200E55B124AAAE5466F7001EE702974B025C8
:1055C2005BF582E4341EAF82F55D8F5E7F101200C0
:1055D20016855E82855D83E0FFA3E0FD126DBE8FBE
:0655E2005CE4FD124F61C4
:0155E80022A0
:024F61008D6B56
:104F630075F020EF900280123A3EAF8285836E8FF8
:104F73006FE0F56CD394004060E56C9410505AE5F3
:104F83006B7014124ACF124AB1504E124A8F124F0D
:104F9300E2056D056D80EFE56B64017019124ACD72
:104FA300124AB15034124A8F124FE2302402802940
:104FB300056D056D80EAE56B6402701D124ACD1222
:104FC3004AB15015124A8FA3E0FD12654530240300
:0E4FD300024DC1056D056D80E67F50126ED156
:084FE10022A3E0FD1265452248
:100D2400855C82855B83A3A3E0FF855C82855B830E
:100D3400A3222430F58274003EF583EDF0AF62EF18
:100D44003395E0FEE55F2FF582E55E3EF58322E50F
:100D5400822406F582E43583F583E0FF126D99ADB4
:100D640007AF63EF3395E0FEEF22A3A3E0FFE55C5A
:100D74002404F582E4355BF583E022E55F2405F580
:100D840082E4355EF583E022E55F2405F582E435EF
:100D94005EF583E0FFE55F2406F582E4355EF583C6
:100DA400E0228E69F56AAF68EF3395E0FEE5662FC1
:100DB400F582E5653EF583222455F582E4340AF58F
:100DC40083EFF0E56275F007A422AF60EF3395E09E
:100DD400FEE56175F008900158123A3EE5822FF560
:100DE40082E5833EF58322E5662405F582E43565D4
:100DF400F583E022E55E75F007A42454F582E4341B
:100E04000AF58322A3A3A3E0FF8D828C83E58224C9
:100E140004F582E43583F583E022E55E75F007A4EA
:100E24002451F582E4340AF5832224E0F582740A1D
:100E34003EF583E5822DF582E5833CF58322E55E6C
:100E440075F007A42453F582E4340AF58322E55FA0
:100E54002405F582E4355EF583E0FFE55F2406F5BD
:100E640082E4355EF583E022E55E75F007A4245242
:100E7400F582E4340AF58322749F2562F582E43412
:100E840000F58322746F2562F582E43400F5832231
:100E94002450F582E4340AF58322ECFF3395E0FE16
:100EA400EF25E0FFEE33FE75F02022E5602405F522
:100EB40082E4355FF58322D3EF6480948022AB070C
:100EC400AA068B828A83A3A3A3E0FFEB2404F58202
:100ED400E43AF583E0FD228F828E83A3A3A3E0226C
:100EE400855F82855E83A3A322AB5DAD5AAF5CAE02
:100EF4005B22FFE562FD3395E0FCE55F2DF582E5BD
:100F04005E3CF5832233CE33CE92E022A2E0CE13B0
:100F1400CE132275F00AA42DFDE5F03CFCE5662213
:100F2400E5602405F582E4355FF583E022E562752A
:100F3400F008900158023A3EE55E75F007A4245586
:100F4400F582E4340AF583E022AB5AAD5DAF5CAEC2
:100F54005B22EF7C002563FDEC35628D82F58322F4
:100F6400A3A3E0FFAD5A22540FF5657808AF03AE92
:100F740002EF08220564E564AE632275F020123A9C
:100F84003EE0FEA3E0FF22E0FAA3E0FB780CFFAE14
:100F9400020822E0FCA3E0FD7804FFAE040822E589
:100FA400632561F582E43562F58322E5662DF582D9
:100FB400E5653CF58322E5662FF582E5653EF5831C
:100FC400222431F5827400222480F58274023EAF1B
:100FD40082222560F560E4355FF55F2285608285B5
:0D0FE4005F83228F828E83A3A3E0640A2224
:02055B008F5AB5
:10055D00C22AE4F542D223D22D1259E77D4B7F02F8
:10056D001266B87D02E4FF1266B87D32E4FF1266B2
:10057D00B87D607F021266B87D027F07124ED9509A
:10058D00057F04126F12900528E0F536A3E0F537CC
:10059D007F03126F12E55A7006A22492298009E595
:1005AD005AB40104A2259229E53745367005D22AA1
:1005BD00020A223029DFE55A7006A2249229800909
:1005CD00E55AB40104A22592292029EAE55A700BB7
:1005DD00755B1E755C6085455D800EE55AB401093D
:1005ED00755B1E755CB085465DE55DD3940050036B
:1005FD00020A1C855C82855B83E0640B6003020A42
:10060D0017A3E0FFB40A0AE55DB40205D22A020A77
:10061D001CEF6401701E120D2EA3E0640A7015E527
:10062D005D6405700F120D2E120D6E120A4D1231F2
:10063D0024020A1C120D2EE0B40111120D2EA3E09E
:10064D00B40109120EED12171B020A1C120D2EE039
:10065D006401701E120D2EA3E064027015E55D6439
:10066D0005700F120D2E120D6E120A4D1261BA0287
:10067D000A1C120D2EE06401701D120D2EA3E064F4
:10068D00037014E55DB4050F120D2E120D6EFDAB4A
:10069D005A123A70020A1C120D2EE0B4011D120DF1
:1006AD002EA3E0B40415E55DD39405400EAB5AAD11
:1006BD005CAC5BAF5D122FF0020A1C120D2EE064D4
:1006CD0001701D120D2EA3E064057014E55DB405D7
:1006DD000F120D2E120D6EFDAB5A125B25020A1C68
:1006ED00120D2EE06401701D120D2EA3E064067034
:1006FD0014E55DB4050F120D2E120D6EFDAB5A12E1
:10070D004D34020A1C120D2EE0B4011D120D2EA344
:10071D00E0B40715E55DD39405400EAB5AAD5CAC66
:10072D005BAF5D124673020A1C120D2EE064017060
:10073D001D120D2EA3E064087014E55DB4050F12B3
:10074D000D2E120D6EFDAB5A1261F4020A1C120D24
:10075D002EE0B40215120D2EA3E0B40A0DE55DB422
:10076D000308AF5A12637B020A1C120D2EE0B4026D
:10077D0016120D2EA3E0B4010EE55DB40E09120E96
:10078D00EF122D7A020A1C120D2EE0B40216120D74
:10079D002EA3E0B4020EE55DB40709120EEF12525E
:1007AD00DD020A1C120D2EE0B40215120D2EA3E06F
:1007BD00B4090DE55DB40308AF5A125514020A1CB5
:1007CD00120D2EE064027019120D2EA3E0B4091162
:1007DD00E55DB4040C120D2E120F64126787020A28
:1007ED001C120D2EE064037021120D2EA3E0640A7D
:1007FD007018E55D64057012120D2E120D6EFD124E
:10080D006DBEAD5A124728020A1C120D2EE064036C
:10081D007029120D2EA3E064017020E55DD39405BF
:10082D004019120D2E120D6EFD126DBE855A62AB62
:10083D005DAD5CAC5B123DFF020A1C120D2EE06437
:10084D00037021120D2EA3E064027018E55D64059E
:10085D007012120D2E120D6EFD126DBEAD5A125F7D
:10086D00D6020A1C120D2EE0B40315120D2EA3E0B4
:10087D00B4030DE55DB40308AF5A126052020A1CB1
:10088D00120D2EE0B40318120D2EA3E0B40410E5E2
:10089D005DD394034009120F4D1249C3020A1C1275
:1008AD000D2EE0B40315120D2EA3E0B4050DE55D7C
:1008BD00B40308AF5A126DAC020A1C120D2EE0B42F
:1008CD000316120D2EA3E0B4060EE55DB405091254
:1008DD000EEF1268C1020A1C120D2EE0640370198E
:1008ED00120D2EA3E0B40711E55DB4040C120D2E0C
:1008FD00120F64126BCB020A1C120D2EE0B40316FC
:10090D00120D2EA3E0B4080EE55DB40409120EEF2E
:10091D001268E6020A1C120D2EE064057014E55DE6
:10092D00B4040F120D24A3A3E0FDAB5A121F7102E4
:10093D000A1C120D2EE0B40516120D72B40B10E543
:10094D005DD394054009120F4D12337D020A1C121E
:10095D000D2EE064067014E55DB4040F120D24A392
:10096D00A3E0FDAB5A122163020A1C120D2EE0B456
:10097D000616120D72B40B10E55DD39405400912E5
:10098D000F4D122694020A1C120D2EE06409701AE6
:10099D00120D2EA3E0B40A12E55DB4040D120D2E56
:1009AD00A3A3E0FF125DC2020A1C120D2EE0640922
:1009BD007018120D2EA3E0B40110E55DB4040B12F6
:1009CD000D2E120F641262D78045120D2EE0B40960
:1009DD0017120D2EA3E0B4020FE55DD39404400869
:1009ED00120EED1214CD8027120D2EE06409701A2F
:1009FD00120D2EA3E0B40310E55DB4040B120D2E01
:100A0D00120F64125D3080078000AF5A126BE82020
:100A1D002A030205A2C21ED22DAF5A1259E77D60DC
:100A2D007F021266B87D327F031266B87F03126FA4
:0F0A3D0012125E0A7FFF126ED1E47885F6C22393
:080A4C0022FD126DBEAD5A221D
:08171B008E5E8F5F8D608B6113
:10172300120EDBFFE55F2404120D83FD1264508F5C
:101733006274E22562F562C39400500302191CE54A
:10174300629414400302191CE5616406701D120DB6
:101753007FB4010C120DC7120E947401F002191814
:10176300120DC7120E94E4F0021918E561640E60BD
:101773000302183AE55F240C120D83FFB40A14E543
:101783005F240D120D83B40A0A120DC7120E24E44E
:10179300F08013E55F240D120D83FD126C3F120DD3
:1017A300C7120E24EFF0E55F240A120D83FFB40A7B
:1017B30014E55F240B120D83B40A0A120DC7120E2F
:1017C30072E4F08013E55F240B120D83FD126C3F6E
:1017D300120DC7120E72EFF0E55F2409120D83FF9D
:1017E300640A6006EFD39409400A120DC7120E482B
:1017F300E4F08010E55F2409120D83FF120DC71278
:101803000E48EFF0120D7FFFB40B15E55F240612AF
:101813000D83B40B0B120DC7120DFE74FFF080087D
:10182300121948120DFEEFF0121924120DBC120EFC
:10183300947401F0021918E561640A706E120DC701
:10184300120E24E4120DC6120E72E4F0E55F2409B1
:10185300120D83FF640A6006EFD39409400A120D48
:10186300C7120E48E4F08010E55F2409120D83FFD0
:10187300120DC7120E48EFF0120D7FFFB40B15E5E2
:101883005F2406120D83B40B0B120DC7120DFE74E9
:10189300FFF08008121948120DFEEFF012192412FE
:1018A3000DBC120E947401F0021918E561640970FD
:1018B30068120DC7120E24E4120DC6120E72E41242
:1018C3000DC6120E48E4F0120D7FFFB40B15E55F51
:1018D3002406120D83B40B0B120DC7120DFE74FFF9
:1018E300F08013E55F2406120D83FD126C3F120D89
:1018F300C7120DFEEFF0E55F2407120D83FFE55FCE
:101903002408120D83FD126C3F120DC7120DBC1279
:101913000E947401F0D22C8002C22CAF60126EA719
:1019230022E55F2407F582E4355EF583E0FFE55F9A
:101933002408F582E4355EF583E0FD126C3FE56231
:1019430075F007A422E55F2406F582E4355EF5838E
:0C195300E0FD126C3FE56275F007A42275
:103124008F5E8D5FE55ED3941D5003023230E55E01
:1031340094324003023230D22DAF5F1259E77D46FC
:103144007F071266B8AF5E1235A474E2255EF55EA1
:10315400120E20E07021120E6CE0701B120E42E081
:103164007015120DF8E0700F120F3C700A123249FC
:103174007D537F02023226123238E55E75F007A4D1
:10318400120E94E070047D3680027D387F0612664C
:10319400B8123238120E1EE0FFD394014034EF947B
:1031A40013502F7D097F061266B8120E1E1232408C
:1031B4007FF47E01126C5B7D0E7F031266B87D3551
:1031C4007F061266B87D097F061266B8120E6C126D
:1031D40032407FF47E01126C5B120E42E0FF600508
:1031E400125A8A800A1232497D0F7F031266B87D13
:1031F400277F021266B8120DF8E0FFF46008126C23
:10320400FB1235A480077D187F021266B87D377FD4
:10321400041266B8120F3CFF126CFB1235A47D0534
:103224007F061266B8C22DAF5F0259E7C22CAF5FAA
:10323400126EA7227FF47E01126C5B22E0FF126CF7
:0D324400FB1235A4227D187F021266B8220D
:0261BA008D5EF8
:1061BC00EFD3941D402AEF9432502574E22FFFE464
:1061CC00FEEEFD3395E0FCEF75F007A42450F5824C
:1061DC00E4340A120E35E4F00EBE07E5D22C800230
:0761EC00C22CAF5E126EA78A
:0161F3002289
:062D7A008E5E8F5F8D608C
:102D8000D22B120EDBFFE55F2404120D9D122EA143
:102D9000C39418501C855F82855E83A3A3A3E0FFC4
:102DA000E55F2404120D9DFD126D867883A60780D1
:102DB00006E47883F6C22B120D8C122EA1C3943C2C
:102DC000500D120D8CFD126D867884A6078006E4E6
:102DD0007884F6C22BE55F2407120D9DFF126E3931
:102DE0008F61E561D394004017E56194085011E5C7
:102DF0005F2407120D9DFF126E397880A6078006AA
:102E000078807601C22BE55F2408120D9DFFE55FF7
:102E10002409120D9D122EAA401FE561942050191D
:102E2000E55F2408120D9DFFE55F2409120D9DFD4D
:102E3000126D867888A607800678887601C22BE511
:102E40005F240A120D9DFFE55F240B120D9D122ECB
:102E5000AA401FE561940D5019E55F240A120D9DEB
:102E6000FFE55F240B120D9DFD126D867881A6078C
:102E7000800678817601C22BE55F240C120D9DFF40
:102E8000E55F240D120D9DFD126D867882A6073038
:102E90002B07125886D22C8002C22CAF60126EA76C
:102EA00022FD1264508F61E56122FD1264508F6132
:062EB000E561D39400224D
:0652DD008E5E8F5F8D6004
:1052E300D22B120EDBFFE55F2404120E6312534828
:1052F3009418501C855F82855E83A3A3A3E0FFE51A
:105303005F2404120E63FD126D867883A607800660
:10531300E47883F6C22B120E52125348943C500D7C
:10532300120E52FD126D867884A6078006E47884F7
:10533300F6C22B302B07125886D22C8002C22CAF18
:0453430060126EA7DF
:0B53470022FD1264508F61E561C3225B
:106E3900120EBB4008EF6480948A5001227F002221
:106D8600AE05126E39EFC454F0FDAF06126E39EF40
:036D96004DFF228C
:10637B008F5ED22D1259E77D1E7F081266B87D26DF
:10638B007F081266B87D527F041266B8C22B126862
:10639B009B125C9C7880E6FF125A8A125991C22D8F
:0663AB00AF5E1259E7226B
:106787008D5EEFD3940A4006EFD3940F4003EF706A
:106797000E90002BEFF0D22CAF5E126EA7D322C261
:0867A7002CAF5E126EA7C322A5
:025514008F5EA8
:10551600D22D1259E77D207F051266B87D2E7F03B6
:105526001266B87D527F041266B890002BE0F55FD4
:10553600E55FB40B067D5F7F078034E55FB40C063C
:105546007D5E7F068029E55FB40D067D0A7F0280B9
:105556001EE55FB40E067D327F028013E55FB40F51
:10556600067D467F028008E55F70077D0A7F03128D
:0955760066B8C22DAF5E1259E7C0
:01557F002209
:106BCB008D5E120EBB400EEF6480948650071264EC
:0D6BDB001CD22C8002C22CAF5E126EA722CD
:0268C1008D5EEA
:1068C300120EC2126450120EBB4010EF648094A1EA
:1068D3005009900029EFF0D22C8002C22CAF5E1237
:0268E3006EA79E
:0168E5002290
:0268E6008D5EC5
:1068E800120EC2126450120EBB4010EF648094A1C5
:1068F8005009900028EFF0D22C8002C22CAF5E1213
:026908006EA778
:01690A00226A
:106D9900D3EF648094814008EF6480948A50012283
:036DA9007F002246
:106E4900120EBB4008EF648094A15001227F0022FA
:0814CD008E5E8F5F8D608B6164
:1014D500120EDB14F56374FC2561F5616403600F7E
:1014E500E56164076009E561640B60030216B8C332
:1014F500E5636480948050030216B8E563648094C4
:101505008840030216B8E4F562120D657803C3330B
:10151500CE33CED8F92430F58274003EF583AF6220
:10152500EF3395E0FE120DE0E4F00562E562B408E4
:10153500D8756204E56164037029120D411216FE27
:10154500120D637803C333CE33CED8F9120D36A30B
:10155500A3120D5E7803C333CE33CED8F9120FC56F
:101565000216AFE56164077069120D411216FE128D
:101575000D637803C333CE33CED8F9120D36A3A34A
:10158500120D5E7803C333CE33CED8F9120FC512D0
:101595000D3CA3A3A3120D5E7803C333CE33CED87F
:1015A500F92432F5827400120D3C1216C0C333CEF5
:1015B50033CED8F92433F5827400120D3C120D5345
:1015C5007803C333CE33CED8F92434F582740002C0
:1015D50016AFE561640B60030216B8120D41E01207
:1015E5000EF6A3E0FD126450126E49120D637803E6
:1015F500C333CE33CED8F9120D36A3A3120D5E78C0
:1016050003C333CE33CED8F9120FC5120D3CA3A3B5
:10161500A3120D5E7803C333CE33CED8F92432F549
:10162500827400120D3C1216C0C333CE33CED8F9E6
:101635002433F5827400120D3C120D537803C33325
:10164500CE33CED8F92434F5827400120D3CE582F0
:101655002407120D577803C333CE33CED8F924357A
:10166500F5827400120D3CE5822408120E15120E47
:10167500F6E5822409120E15FD126450126E491208
:101685000D637803C333CE33CED8F92436F582748F
:1016950000120D3CE582240A120D577803C333CEA0
:1016A50033CED8F92437F58274003EF583EDF0D2B8
:0A16B5002C8002C22CAF60126EA759
:1016BF0022E5822404F582E43583F583E0FFE562B9
:1016CF00FD3395E0FCE55F2DF582E55E3CF583E5A6
:1016DF00822405F582E43583F583E0FD1264501210
:1016EF006E49AD07AF63EF3395E0FEEF780322E06D
:1016FF00FFE562FD3395E0FCE55F2DF582E55E3C8D
:0C170F00F583A3E0FD126450126E492225
:045D30008D5EAC07D1
:105D3400D3EC648094804035EC64809489502EE4E4
:105D4400FDECFF3395E0FEEF7803C333CE33CED8BA
:105D5400F92428F58274003EF583EDFF3395E0FEC7
:105D6400120DE0E4F00DBD08D8D22C8002C22CAF95
:045D74005E126EA7A6
:015D78002208
:1062D7008D5E120EBB402FEF648094895028EF1417
:1062E700FFE55E24FF922B124FE9D22DAF5E1259C4
:1062F700E77542017F327E00126C5BE54270FCC29B
:076307002DAF5E1259E722E1
:084673008F5E8C5F8D608B618E
:10467B00856082855F83120E08FD1264508F62E5A0
:10468B0062D394005003024720E562943240030248
:10469B004720E55E64067036D22DAF611259E77D77
:1046AB00527F051266B8AF621235A4120F24B40103
:1046BB000A120E7C7401F07D388007120E7CE4F038
:1046CB007D367F061266B8C22DAF610259E7E560F1
:1046DB002406120F28640B703C120F24B40108122D
:1046EB000E7C7401F08005120E7CE4F074F9255EEB
:1046FB00F55E75F004123984AFF0EF7014E56024A9
:10470B0006FBE4355FFAAD62E4FF1234A4D22C80D1
:0C471B0006C22C8002C22CAF61126EA7F7
:01472700226F
:082FF0008F5E8C5F8D608B6128
:102FF800856082855F83120E08FD1264508F62E53A
:1030080062D39400500302311CE562942840030205
:10301800311CE55E64067037D22DAF611259E77D29
:10302800527F051266B8AF621235A4120EAFE0B433
:10303800010A120E887401F07D388007120E88E4A8
:10304800F07D367F061266B8C22DAF610259E7E5FA
:10305800602406120EB3E0640B600302311C120EEA
:10306800AFE0B40108120E887401F08005120E88D2
:10307800E4F0E4FFFEE5602407120EB3E5822E12A9
:103088000E15B40B04AF0680040EBE08E8EF7003FB
:1030980002311CC39408507C120F31EFF07E01EF0F
:1030A8002401FDE433FCEEC39DEC6480F874809841
:1030B8005020E5602406120EB3E5822E120E15FD8F
:1030C800120F31E5822EF582E43583F583EDF00E9B
:1030D80080CDE5602408120EB3E5822F120E156428
:1030E8000B602DEF2408FEC3E55E9EF55E75F004C7
:1030F800123984AEF0EE701CE5602407FDE4355FFC
:10310800FC7E00ED2FFBEE3CFAAD627F011234A489
:0B311800D22C8002C22CAF61126EA707
:013123002289
:0834A4008F638D648A658B665D
:1034AC00756801E4F567120DAAE0FF6409703E121D
:1034BC0035958003120F09D8FB120DA612358778AB
:1034CC0008EF088003120F09D8FB120DA6A3A3E086
:1034DC00FFE568FD3395E0FCE5662DF582E5653C7E
:1034EC00F583A3A3A3E0FD126DBE023540120DAA15
:1034FC00E0FF1235958003120F09D8FB120DA612AE
:10350C0035877804EF088003120F09D8FB120DA63B
:10351C00A3A3E0FF126F08EF426AAE69AF6A7804AA
:10352C00EF088003120F09D8FB120DA6A3A3A3E08A
:10353C00FF126F08EF426AE563700FAF67120D67F9
:10354C00120EA5E564900AC08012E563B40117AFB2
:10355C0067120D67120EA5E564900530120DDDE5BE
:10356C0069F0A3E56AF074042568F5680567C3E59E
:0A357C00676480949050030234B29B
:1035860022A3E0FF126F08EF426AAE69AF6A221209
:0E3596006F087569008F6AAE697804EF08222D
:0A6F0800EFD3940940037F0022221A
:023A70008B5E6B
:103A72001264508F61E561D394005003023B52E51A
:103A82006194334003023B52D22DAF5E1259E77D5F
:103A9200527F051266B8AF611235A4746F256112A8
:103AA2000E8CE060047D3880027D367F061266B897
:103AB2007F2C7E01126C5BE561120F33E0F55F70C3
:103AC200077D1B7F061266B87D577F021266B8E536
:103AD2005F603B756001AF5F120D672401FFE43E3A
:103AE200FEAD60ED3395E0FCC3ED9FEE6480F8EC33
:103AF2006480985019120DCEE0B40A04E4FD8006E9
:103B0200120DCEE0FDE4FF1266B8056080C87F2C7E
:103B12007E01126C5BE561900530120F7F90000010
:103B2200EEF0A3EFF04E70077D1B7F061266B87DA4
:103B32000C7F031266B8900000E07002A3E06009F7
:103B4200E56114FD7F01122ADCC22DAF5E0259E746
:073B5200C22CAF5E126EA74A
:013B59002249
:024D34008B5E94
:104D36001264508F5FE55FD394004077E55F94334C
:104D46005071D22DAF5E1259E77D527F051266B8BB
:104D5600AF5F1235A4749F255F120E80E060047D5C
:104D66003880027D367F061266B87F2C7E01126C73
:104D76005B7F2C7E01126C5BE55F900AC0120F7F91
:104D8600900000EEF0A3EFF04E70077D1B7F061239
:104D960066B87D0C7F031266B8900000E07002A32F
:104DA600E06009E55F14FDE4FF122ADCC22DAF5E68
:0A4DB6000259E7C22CAF5E126EA78F
:014DC00022D0
:0261F4008B5EC0
:1061F600126450AD07EDD394004025ED9433502042
:10620600E4FC120E9EED900AC0120DDDE4F0A3F040
:106216000CBC10EE749F2D120E80E4F0D22C80027E
:07622600C22CAF5E126EA74F
:01622D00224E
:025B25008B5E95
:105B2700126450AD07EDD394004036ED94335031F5
:105B3700E4FC120E9EED900530120DDDE4F0A3F0AB
:105B47000CBC10EE746F2D120E8CE4F0FCECFF33DE
:105B570095E0FEED120DD7E4F00CBC08F0D22C80D6
:085B670002C22CAF5E126EA712
:015B6F002213
:042ADC008F628D6315
:102AE000E4F564E5627052AF64120D6725E0FDEE17
:102AF00033FCAF63120D677805C333CE33CED8F9FC
:102B0000120E2E120F8B8003120F10D8FB120F6BB8
:102B10008003120F10D8FB540FF566AF63120D67D8
:102B20007805C333CE33CED8F9120E2E120F97800C
:102B300003120F10D8FB022B9AE56264017064AF98
:102B400064120D6725E0FDEE33FCAF63120D67786C
:102B500005C333CE33CED8F92450F5827405120E56
:102B600034120F8B8003120F10D8FB120F6B8003EF
:102B7000120F10D8FB540FF566AF63120D6778057E
:102B8000C333CE33CED8F92450F5827405120E34F7
:102B9000120F978003120F10D8FB540FF567ED54F6
:102BA0000FF568E565700CE5667008E5677004E58B
:102BB00068607CAD65E4FF1266B8AD66E4FF12663E
:102BC000B8E56564097045856769AF69FE7804EF0B
:102BD000088003120F09D8FBF569E5684269E569C9
:102BE000B4990B7D09E4FF1266B87D098027E56979
:102BF00075F00A84F56AFDE4FF1266B8E56A75F0BF
:102C00000AA4FFC3E5699FF56AFD8009AD67E4FF8B
:102C10001266B8AD68E4FF1266B87FF47E01126CEC
:0F2C20005B0564C3E564648094A05003022AE35B
:012C2F002282
:10645000EFD394004015EF940B5010EFC3940A5003
:1064600008EF75F00AA4FE8002E4FEEDD39400402C
:106470000EED940B5009EDC3940A5003ED2EFEAFC0
:016480000615
:0164810022F8
:0649C3008E5E8F5F8B6029
:1049C900756105756240D3ED64809484407CED6423
:1049D9008094A55075ED24FDF563D39404406BE5EF
:1049E9006320E06613F5640562E562AE6170020555
:1049F9006114F5828E83E564F07403255FF55FE445
:104A0900355EF55EE4F563E563C395645033855F10
:104A190082855E83E0FFA3E0FD126DBE0562E5625B
:104A2900AC617002056114F5828C83EFF0055FE5D6
:104A39005F7002055E055FE55F7002055E056380D4
:104A4900C6D22CAF60126EA7D322C22CAF60126EF1
:024A5900A7C3F1
:014A5B002238
:043DFF008C5F8D60E8
:103E0300120EBB5003023ED7EF6480949540030229
:103E13003ED7EB648094875003023ED7EB648094D3
:103E2300E44003023ED7120D677805C333CE33CE89
:103E3300D8F9120FCCF5638F64EB24FBF565D394AB
:103E4300025003023ED7E56575F00384E5F0600395
:103E5300023ED7E56575F00384F567C3941050748B
:103E6300120F787002056314F5828E83E567F07490
:103E730005120FD6E4F565E565C395675052120F39
:103E8300E0E0F566B40A10120F787002056314F5CA
:103E9300828E83E4F0800F120F787002056314F5AD
:103EA300828E83E566F0120FE0A3E0FF120FE0A31A
:103EB300A3E0FD126DBE8F66120F787002056314C6
:103EC300F5828E83E566F07403120FD6056580A72D
:0B3ED300D22C8002C22CAF62126EA73E
:013EDE0022C1
:082694008E5E8F5F8D608B618B
:10269C00C22B120FE7600302273112280C500302E1
:1026AC00272CE5649408E56394075074C3E56064D3
:1026BC0080948A506B120EE4A3E0F562B40106908C
:1026CC000520022781E562B40206900522022781CB
:1026DC00E562B40306900524022781E562B4040682
:1026EC00900526022781E562B4050690052802278D
:1026FC0081E562B4060690052A022781E562B407DB
:10270C000690052C022781E562B4080590052E8001
:10271C0064E562B40905900530805AD22B0227FD7E
:10272C00D22B0227FD120EE4E064017052AD60AFB3
:10273C005FAE5E12280C50030227FDE5649408E599
:10274C0063940740030227FDC3E5606480948A40CC
:10275C00030227FD120EE4A3E0F562B40A0590050E
:10276C00328012E562B401059005348008E562B44C
:10277C000209900536E563F0A3806FD22B807212AC
:10278C000EE4E06402706AAD60AF5FAE5E125B7027
:10279C007563008F64C3E5649463E56394005051E2
:1027AC00C3E560648094885048120EE4A3E0F5629F
:1027BC00B40107900538EFF08037E562B40205905C
:1027CC0005398026E562B4030590053A801CE56264
:1027DC00B4040590053B8012E562B4050590053CF8
:1027EC008008E562B4060890053DE564F08002D2ED
:0F27FC002B302B04C22C8002D22CAF61126EA79F
:10280B002212487C8E638F64D3E564943BE563941A
:02281B00002299
:06487C008E658F66A905A0
:104882007D057C00120FAFE0C3940A4005120FAF02
:10489200E4F00DBD00010CED640A4C70E7B90607A7
:1048A200120DEBFF7E0022E964077010120DEB750A
:1048B200F00AA4ACF0FDE5662406801BE9640870EA
:1048C20021120DEB75F064A4ACF0FDE5662406122E
:1048D2000DEF120F172407120DEF2DFDE43CAF056B
:1048E200FE22E964097033120DEBFF7E007C037D2A
:1048F200E81239A6AC06AD07E5662406120DEF757F
:10490200F064120F1A2407120DEF120F1724081267
:0D4912000DEF2DFDE43CFEAF0522E4FEFF9D
:01491F002275
:065B70008E658F66A90599
:105B76007F057E00120FBAE0C3940A4005120FBAE1
:105B8600E4F00FBF00010EEF64084E70E7E964070A
:105B96007020E5662405F582E43565F583E075F049
:105BA6000AA4FFE5662406F582E43565F583E02F51
:045BB600FF227F004B
:015BBA0022C8
:08337D008E5E8F5F8D608B6195
:10338500C22BD3E56064809484500302342BE5603E
:103395006480948D400302342B120FE760030234DE
:1033A5002B120EDB123A4A33CB0133D60233E1033B
:1033B50033EB0433F50533FF0634090734130834BA
:1033C5001D0900003427756201756300D22B023494
:1033D50062756201756308D22B02346275620175EC
:1033E5006310D22B8077756201756318D22B806DBF
:1033F500756201756320D22B806375620175632840
:10340500D22B8059756201756330D22B804F75625E
:1034150001756338D22B8045756201756340D22BE7
:10342500803BC22B8037D3E56064809484402EE5D1
:10343500606480948D5026855F82855E83A3A3E0BA
:10344500B4011A855F82855E83A3A3A3E024F67089
:103455000A756201756358D22B8002C22B302B3757
:10346500E4FF120F56E4F00FBF08F7E56024FB8573
:103475006382856283F07F01E55F2404F582E4358C
:103485005EF583E5822F120E15FE120F56EEF00F34
:0E349500BF08E5D22C8002C22CAF61126EA7D8
:0134A3002206
:044728008F5E8D5FB4
:10472C00E55ED3940050030247CBE55E941540033D
:10473C000247CBD22DAF5F1259E77D5F7F05126622
:10474C00B8AD5EE4FF1266B87D527F041266B87F86
:10475C00F47E01126C5B75F020E55E900280123ADB
:10476C003EAF828583628F63E0F560603DD3940039
:10477C004046E56094105040E56025E0F5607561B9
:10478C0001E5602401FFE433FEC3E5619FEE648024
:10479C00F87480985022120FA3E0FF120FA3A3E02D
:1047AC00FD1265450561056180D77D1B7F0612668C
:1047BC00B87D5F7F051266B8C22DAF5F0259E7C2A4
:0647CC002CAF5F126EA786
:0147D20022C4
:102163008F5E8D5F8B60E55E640A7074E55FC39478
:102173000A40030222D0122306E4FDFF1266B8AD23
:102183005F1222DFE55F123A4A21AB0121B102213E
:10219300B70321BD0421C30521C90621CF0721D5DA
:1021A3000821DB09000021E090052002222A900586
:1021B3002202222A90052402222A90052602222A9C
:1021C30090052802222A90052A02222A90052C0231
:1021D300222A90052E02222A900530804A0222C923
:1021E300E55E64017052E55FD394004006E55F94B9
:1021F300034006E55F640A703C122306E55FB40AF8
:102203000A7D0A1222DF900532801CE55FB4010AC1
:102213007D0B1222EC900534800DE55FB402137D33
:102223000C1222EC900536E0FEA3E0FF1264B40228
:1022330022D70222C90222D0E55E64026003022291
:10224300D7E55FD3940050030222D0E55F94075093
:102253007CD22DAF601259E77D277F081266B87DC7
:1022630006E4FF1266B87D14E4FF1266B8E55F2446
:10227300FE601A14602114602814602F1460362441
:102283000570437D011222F990053880307D0212DA
:1022930022F990053980267D0312231C90053A808C
:1022A3001C7D0412231C90053B80127D05122329FB
:1022B30090053C80087D0612232990053DE0FF7EB2
:1022C300001264E5800EAF60126BE88007C22CAF8A
:1022D30060126EA7C22DAF601259E722E4FF1266A7
:1022E300B87D527F041266B822E4FF1266B87D52AD
:1022F3007F041266B822E4FF1266B87D527F04128F
:1023030066B822D22DAF601259E77D277F08126687
:10231300B87D06E4FF1266B822E4FF1266B87D5268
:102323007F041266B822E4FF1266B87D527F04125E
:0323330066B82267
:044AF4008E638F64DA
:104AF8000564E5647002056314F5828E83E0F5664B
:104B0800607AC3940850757F2C7E01126C5BE4F5C3
:104B180065E565C395665064856482856383E012A4
:104B28003A4A4B65004B430A4B470B4B4D0C4B53D2
:104B38000D4B590E4B5F0F00004B6BE4FD802D7D34
:104B48005F7F0780287D5E7F0680227D0A7F028046
:104B58001C7D327F0280167D467F0280107D0A7F91
:104B680003800A856482856383E0FDE4FF1266B8EA
:0C4B78000564E564700205630565809526
:014B8400220E
:061F71008F5E8D5F8B60A6
:101F7700C22BE55E640A6003022065E55F123A4AF8
:101F87001FA6011FB9021FCC031FDF041FF2052084
:101F97000806201E07203408204909000020611286
:101FA700209A7D011220E8756101756200D22B022B
:101FB700208112209A7D021220E87561017562085E
:101FC700D22B0220811220B67D031220F575610104
:101FD700756210D22B0220811220B67D041220F5E3
:101FE700756101756218D22B0220811220D212214D
:101FF700487D05122118756101756220D22B0220D8
:10200700811220D21221487D0612211875610175AF
:102017006228D22B02208112210212215C7D071235
:102027002125756101756230D22B022081122102B0
:1020370012215C7D08122125756101756238D22B4A
:102047008038122132E4FDFF1266B87D0912214F54
:10205700756101756240D22B8020C22B801CE55E22
:1020670064017016E55F24F670101221327D0A12A2
:10207700214F756101756258D22B302B09AF62AEC3
:1020870061124AF48005AF60126BE8C22DAF60128F
:0220970059E707
:1020990022D22DAF601259E77D577F021266B87DB3
:1020A90005E4FF1266B8E4FDFF1266B822D22DAF2F
:1020B900601259E77D577F021266B87D05E4FF1269
:1020C90066B8E4FDFF1266B822D22DAF601259E757
:1020D9007D577F021266B87D05E4FF1266B822E4D7
:1020E900FF1266B87D527F041266B822E4FF1266B9
:1020F900B87D527F041266B822D22DAF601259E71B
:102109007D577F021266B87D05E4FF1266B822E4A6
:10211900FF1266B87D527F041266B822E4FF126688
:10212900B87D527F041266B822D22DAF601259E7EA
:102139007D577F021266B87D05E4FF1266B822E476
:10214900FDFF1266B822E4FF1266B87D527F0412C1
:0A21590066B822E4FDFF1266B8220A
:1035A4008F72E572D3945940107D5A12368B24A63B
:1035B400FD700302368A023685E572D3944F4016B5
:1035C400E572945A50107D5012368B24B0FD70036E
:1035D40002368A023685E572D394454016E5729424
:1035E4005050107D4612369324BAFD700302368A79
:1035F400023685E572D3943B4012E5729446500C32
:103604007D3C12369324C4FD607C8075E572D394AE
:10361400314012E572943C500C7D3212369B24CE1C
:10362400FD6063805CE572D394274012E5729432A6
:10363400500C7D2812369B24D8FD604A8043E572E5
:10364400D3941D4016E572942850107D1EE4FF1299
:1036540066B8E57224E2FD602D8026E572D39413EA
:103664004016E572941E50107D14E4FF1266B8E50E
:103674007224ECFD60108009E572C394145007AD08
:1036840072E4FF1266B822E4FF1266B8E57222E41F
:0F369400FF1266B8E57222E4FF1266B8E57222F3
:1059E7008F6AE56A700C302D097F01126F257FC021
:1059F700801FE56A700C202D097F01126F127FC08E
:105A07008026E56AB40112302D0F7F02126F257FC1
:105A170030120016C22F02699DE56AB40114202DC9
:105A2700117F02126F127F30126ED17FC87E001273
:035A37006C5B2283
:106979008F69D22D1259E77D607F021266B87D3288
:106989007F061266B87D1E7F051266B8C22DAF69F3
:046999001259E72286
:106BE8008F69D22D1259E77D607F021266B87D3019
:0D6BF8007F031266B8C22DAF691259E72263
:0E6EA7008F68302C03026979AF68126BE82205
:105DC200EF24FE60101460162402701C7F01126F13
:105DD200257F8080107F02126F257F2080077F033E
:105DE200126F257FA01200167FF47E01126C5B7584
:105DF2004204E54270FC7F647E00126C5B7F0312FA
:085E02006F127FA0126ED12285
:1064E5008E618F627C007D0A1239B8AD07E4FF1218
:1064F50066B87D5B7F061266B8AE61AF627C007DD3
:106505000A1239B8E4FF1266B87D4A7F070266B8F9
:0464B4008E618F6204
:1064B8007C007D3C1239B81235A47D057F06126632
:1064C800B8AE61AF627C007D3C1239B8ED4C600C0F
:0C64D800AF051235A47D4A7F071266B89C
:0164E4002295
:025FD6008D5EDE
:105FD800120EBB402FEF648094955028120D6778FD
:105FE80005C333CE33CED8F9120FCCFEE4FD0FEF44
:105FF800AA0670010E14F5828A83E4F00DBD20EE26
:0B600800D22C8002C22CAF5E126EA7EB
:01601300226A
:106052008F5E900540E0D394024015D22D1259E78D
:106062007542037F327E00126C5BE54270FC801544
:10607200D22DAF5E1259E77D1B7F061266B87D0CEA
:0D6082007F031266B8C22DAF5E1259E722EF
:106DAC007E10900540E4F0A3DEFC7E10D22C126E17
:016DBC00A72F
:016DBD0022B3
:106DBE00BF0A02E4FFBD0A02E4FDEF75F00AA42D3E
:026DCE00FF22A2
:106C3F00EFD394094002E4FFEDD394094002E4FD41
:0C6C4F007804EF08800123D8FD4DFF22DF
:1040890007010203040506070707060504030201E1
:1040990003010A0A030307050303020503020A0AC7
:1040A90004050A0A0104050A0A0A04050A0A0203A0
:1040B900070A0A03040A0A04024B00020032072E07
:1040C90003024B0002003202055F000302055F0094
:1040D9000402055F000502055F000604072E082695
:1040E9000640033204072E08260640025304081E20
:1040F90008260452010008024B00020032072E086C
:104109001E08260452010003072B02350636030751
:104119002B0235063803072B0235072603072B0226
:1041290035025302055F000F02055F001002055FAB
:10413900001102055F001202055F001302055F000E
:0A41490014080C0A1D020500241BD7
:105264007461F0A37420F0A37452F0A37401F0A34A
:1052740022A3F0A37461F0A37440F022F0A374039A
:10528400F0E4A3F0A37410F0A37403F0E4A3F0A378
:10529400227461F0A37441F0A3227461F0A3F0A31B
:1052A4007430F0A3227496F0A37432F0A37495F0D2
:1052B400A3741EF0A322F0A37461F0A314F0A374EA
:1052C40070F0A3E4F022A3F0A37452F0A3223CF5FF
:0952D40083E0FEEF3395E0FC22BB
:10003E007E407F897C017D507B08125ED47E407F9E
:10004E00917C017D587B08125ED47E407F997C01A5
:10005E007D007B04125ED47E407FA57C017D087BF3
:10006E0004125ED47E407FA17C017D107B04125E63
:10007E00D47E407F9D7C017D187B04125ED47E4031
:10008E007FAE7C017D207B05125ED47E407FA97CF5
:10009E00017D287B05125ED47E407FB37C017D30CE
:1000AE007B05125ED47E407FB87C017D387B0412C6
:1000BE005ED47E407FBC7C017D407B04125ED47E8C
:1000CE00407FC07C027DA07B09125ED47E407FC93A
:1000DE007C027DC07B07125ED47E407FD07C027D89
:1000EE00E07B05125ED47E407FD57C037D007B05D0
:1000FE00125ED47E407FDA7C037D207B05125ED4B7
:10010E007E407FDF7C037D407B05125ED47E407F88
:10011E00E47C037D607B09125ED47E407FED7C0320
:10012E007D807B09125ED47E407FF67C037DA07BB2
:10013E0009125ED47E407FFF7C037DC07B11125E70
:10014E00D47E417F107C037DE07B07125ED47E411E
:10015E007F177C047D007B07125ED47E417F1E7C60
:10016E00047D207B07125ED47E417F257C047D407A
:10017E007B07125ED47E417F2C7C047D607B051252
:10018E005ED47E417F317C047D807B05125ED47E01
:10019E00417F367C047DA07B05125ED47E417F3B81
:1001AE007C047DC07B05125ED47E417F407C047D45
:1001BE00E07B05125ED47E417F457C057D007B058C
:1001CE00125ED47E417F4A7C057D407B09125ED44F
:1001DE009000297417F07F0312641C900028741984
:1001EE00F090002074B1F09000217491F0900022F4
:1001FE007403F0900023747FF090002404F09000BC
:10020E00257403F0E4900026F0900027F090003063
:10021E0074091252807415F0A37403F0A3741512AE
:10022E0052807409F0A37403F0E4FFEFFD3395E000
:10023E00FC74302DF58274001252D274102DF5829A
:10024E0074003CF583EEF00FBF08E0E4FFEFFD33E2
:10025E0095E0FC74382DF58274001252D274182D6C
:10026E00F58274003CF583EEF00FBF08E090052098
:10027E00E4F0A374B4F0900522E4F0A374B4F0900B
:10028E0005247401F0A374E0F0900526E4F0A37445
:10029E0078F09005287402F0A37458F090052AE4C3
:1002AE00F0A3743CF090052C7402F0A37458F07413
:1002BE000790052EF0A3F0900530F0A3F0900532D4
:1002CE00F0A3F0900534F0A3F0900536E4F0A3749B
:1002DE003CF0900538740AF09005397428F09005BA
:1002EE003A7405F090053B740AF090053CF09005C9
:1002FE003D7428F09000A47401F0900B607415F01A
:10030E00A37411F09000A57401F0900B807415F099
:10031E00A37410F09000A67401F0900BA07415F069
:10032E00A37421F09000A77401F0900BC07415F027
:10033E00A37420F09000A87401F0900BE07415F0F7
:10034E00A37431F09000A97401F0900C007415F0B4
:10035E00A37430F09000AA7401F0900C207415F084
:10036E00A37441F09000AB7401F0900C407415F042
:10037E00A37440F09000AC7401F0900C60745312B2
:10038E00526E743612526E7438F0A3E4F0A37453A6
:10039E00F0A3E4F09000AD04F0900C807453125270
:1003AE006E7434F0A37421F0A37453F0A3E4F090B0
:1003BE0000AF04F0900CC012526C7430F074031243
:1003CE0052CAE4F09000B004F0900CE012526C743B
:1003DE0030F074041252CAE4F09000B104F0900DA3
:1003EE0000125264743212526E7452F0A37420F0E2
:1003FE009000B27401F0900D201252647432F0A38A
:10040E0074021252CB7420F09000B37401F0900D70
:10041E0040745312526E7433F0A3E4F09000B4049F
:10042E00F0900D601252957430F074021252759065
:10043E0000B57401F0900D801252957430F0740571
:10044E001252759000B67401F0900DA01252957470
:10045E0030F0A374061252769000B77401F0900D2E
:10046E00C01252951252A97498F0A3744B12527680
:10047E009000B87401F0900DE01252951252A974CA
:10048E0093F0A374181252769000B97401F0900E86
:10049E00001252957430F0A37413125276A3747036
:1004AE00F0A37402F09000BA14F0900E2012529E37
:1004BE007412F0A3747012526E7461F0A314F09063
:1004CE0000BB7401F0900E4012529E74111252BA7B
:1004DE009000BC04F07461900E601252A07414125D
:1004EE0052BA9000D104F09011001252957492F00D
:1004FE00A3744BF0A37490F0A37402F0A37490F065
:10050E00A37432F07499A3F0A3F0A3746012526E28
:10051E00749112526E7491F0A3E412527690000F01
:10052E007401F0125E0A7F01126F257F40120016D1
:10053E007D2F7F071266B87D0C7F031266B87D3261
:0C054E007F061266B87D1E7F051266B89D
:01055A00227E
:0A5ED4008E5A8F5B8C5C8D5D8B5E37
:105EDE00E4F9C3E55E6480F8E96480985028E9FF30
:105EEE003395E0FEE55B2FF582E55A3EF583E493AC
:105EFE00FFE9FD3395E0FCE55D2DF582E55C3CF5B3
:065F0E0083EFF00980CCD6
:015F1400226A
:10564F00AF6AEF3395E0FEE56975F008A42428F5FD
:10565F0082E43400F583E5822FF582E5833EF583FE
:10566F00E0FFE56AFD3395E0FC22AB66AD65AF6404
:10567F00223EF583E0FD74B82FF582741D3EF5834D
:10568F00EDF0056AE56A22EF3395E0FEEF25E0FFC6
:10569F00EE33FE22A2E0CE13CE13223CF583EFF0C1
:0556AF00056AE56A2216
:045BBB008C5B8D5C16
:105BBF00EF6043D201D202D20CE4F55D855C8285A1
:105BCF005B83E0FEA3E04E6027AF5D125696E55C67
:105BDF002FF582E55B3EF583E0FEA3E0FF1245065D
:105BEF00922920290B055DC3E55D6480949040CC1C
:065BFF00C201C202C20C4B
:015C0500227C
:045C06008C608D61C0
:105C0A00EF6043D201D202D20CE4F562856182854B
:105C1A006083E0FEA3E04E6027AF62125696E5610C
:105C2A002FF582E5603EF583E0FEA3E0FF1245060C
:105C3A00922D202D0B0562C3E5626480949040CCBE
:065C4A00C201C202C20CFF
:015C50002231
:04450600AD07AC064B
:10450A00C22E780CEF0880031256A3D8FB540FF57D
:10451A00637808AF05AE04EF0880031256A3D8FBF0
:10452A00540FF5647804AF05AE04EF088003125601
:10453A00A3D8FB540FF565ED540FF566E56360717A
:10454A00B40108125679123C3D8066E563B402084C
:10455A00125679126B538059E563B40308125679DF
:10456A00123896804CE563B40408125679126AF43C
:10457A00803FE563B405081256791224E68032E5D5
:10458A0063B4060812567912125F8025E563B407F0
:10459A0008125679125AD98018E563B408081256D7
:1045AA007912582B800BE563B40906125679126901
:0345BA000BA22E23
:0145BD0022DB
:103C3D008F678D688B69E567B40113900020E0FFF5
:103C4D001258E1900020EFF0FD7F20023CFAE5676D
:103C5D00B40211900021123D00900021EFF0FD7F84
:103C6D0021023CFAE567B40311900022123D009049
:103C7D000022EFF0FD7F22023CFAE567B4041090BC
:103C8D000023123D0A900023EFF0FD7F23805EE5B7
:103C9D0067B40516900024123D0A900024EFF0FD44
:103CAD007F247E001263B1026515E567B40610909E
:103CBD000025123D14900025EFF0FD7F25802EE5A7
:103CCD0067B40710900026123D14900026EFF0FD0A
:103CDD007F268019E567B40819900027E0FFAB69CE
:103CED00AD681258E1900027EFF0FD7F277E00129E
:103CFD0063B122E0FFAB69AD681258E122E0FFAB82
:103D0D0069AD681258E122E0FFAB69AD681258E168
:013D1D002283
:1058E100D22FAC07BD01047E018033BD02047E02CC
:1058F100802CBD03047E048025BD04047E08801E27
:10590100BD05047E108017BD06047E208010BD07F2
:10591100047E408009BD08047E808002C22FBB0145
:1059210005EE4204800BEB7006EEF452048002C2D5
:075931002F302F03AF042209
:01593800224C
:026B53008B674E
:106B5500C22FEF7016ED7013E5677003025C9CE5BC
:0B6B650067B401077880E6FF125A8A2F
:016B70002202
:063896008F678D688B694D
:10389C00E567700712397CE4FD801AE567B401070F
:1038AC0012397C7D01800EE567B4020CAD69AF68FE
:1038BC00126EB57D02024F61E567B40306124DC16D
:1038CC00C21E22E567B40415AD69AF681264508F4F
:1038DC0043754205E542700302397B80F7E5676466
:1038EC00067017E5687013F56A12564F74102DF5B3
:1038FC008274001256AAB408F022E56764077017A8
:10390C00E5687013F56A12564F74182DF582740021
:10391C001256AAB408F022E56764087027E56870AF
:10392C0023E569701FF56AAF6AEF3395E0FE7410FA
:10393C002FF5827400125680B408EC754201E542F2
:10394C00602D80FAE56764097025E5687021E569EA
:10395C00701DF56AAF6AEF3395E0FE74182FF5828F
:0F396C007400125680B408EC754201E54270FCFD
:09397B0022AD69AF68126EB5229D
:106AF4008F67AE03AF05E567D394004012E5679452
:106B040007500CAD06126EB5AD07AF6712670C22C5
:1024E6008F678D688B69E5677018E5687014E56914
:1024F60070057F01126ED1E56964016003022693BF
:102506008043E567701CE568B40117E56970057FCF
:1025160004126ED1E569640160030226937F04020A
:102526002690E5677029E56864027023E569700501
:102536007F05126ED1E5696401600302269390005F
:102546000FE0B403057F010226907F05022690E581
:1025560067B4011BE5687017E56970057F02126EA6
:10256600D1E569640160030226937F02022690E5A5
:1025760067B4011CE568B40117E56970057F0812A8
:102586006ED1E569640160030226937F08022690F6
:10259600E56764017029E56864027023E5697005E2
:1025A6007F0A126ED1E569640160030226939000EA
:1025B6000FE0B403057F020226907F0A022690E50B
:1025C60067B4021BE5687017E56970057F40126EF7
:1025D600D1E569640160030226937F40022690E5F7
:1025E60067B4021CE568B40117E56970057F10122F
:1025F6006ED1E569640160030226937F100226907E
:10260600E56764027024E5686402701EE56970057A
:102616007F50126ED1E5696401707290000FE0B4CC
:1026260003047F4080647F508060E567B40317E54C
:10263600687013E56970057F80126ED1E5696401E3
:10264600704B7F808044E567B40318E568B40113D6
:10265600E56970057F20126ED1E5696401702E7FF1
:10266600208027E56764037024E5686402701EE530
:102676006970057FA0126ED1E569B4011090000F54
:0E268600E0B403047F8080027FA012001622C1
:10125F008F678D688B69E5677017AD69AF68126E20
:10126F00B58E348F35D3E5359400E534940050F5C1
:10127F0022E567B4011BE568B40116E5697007C282
:10128F00307F01122EB6E569640160030214CC8031
:10129F0058E5676401702BE56864027025E5697095
:1012AF0007C2307F02122EB6E56964016003021493
:1012BF00CC90000FE0640370030214CCD2307F0295
:1012CF008031E5676401702EE56864037028E56975
:1012DF007007C2307F03122EB6E569640160030206
:1012EF0014CC90000FE0B40306D2307F018004D2FB
:1012FF00307F03022EB6E5676401702DE568640444
:10130F007027E569700CC2307F01122EB67F401234
:10131F006ED1E569640160030214CCD2307F0112F3
:10132F002EB67F40120016807CE5676401703AE5A7
:10133F006864057034E569700CC2307F02122EB6F6
:10134F007F10126ED1E569640160030214CC900026
:10135F000FE0640370030214CCD2307F02122EB65A
:10136F007F10120016D22F803EE5676401703BE5B7
:10137F006864067035E569700CC2307F03122EB6B3
:10138F007F50126ED1E569640160030214CCD23034
:10139F007F03122EB690000FE0B403047F4080024B
:1013AF007F50120016C22F02699DE56764027029F3
:1013BF00E56864017023E56970057F100214B3E5D9
:1013CF0069B401057F100214BDE569640260030270
:1013DF0014CCD22F7F010214C9E56764027029E58E
:1013EF006864027023E56970057F200214B3E56914
:1013FF00B401057F200214BDE56964026003021485
:10140F00CCD22F7F020214C9E56764027029E56808
:10141F0064037023E56970057F400214B3E569B476
:10142F0001057F400214BDE569640260030214CC1C
:10143F00D22F7F030214C9E56764027023E5686445
:10144F0004701DE56970047F808059E569B401045B
:10145F007F80805AE56964027063D22F7F04805ABF
:10146F00E56764027023E5686405701DE569700423
:10147F007F048030E569B401047F048031E569643D
:10148F0002703AD22F7F058031E5676402702EE536
:10149F0068640670287D017F07124ED9401FE569E9
:1014AF0070057F08026F12E569B401057F08026FAE
:0E14BF0025E569B40207D22F7F0612297E228E
:025AD9008B67D9
:105ADB00EF7037ED7034E567700690000F0480208F
:105AEB00E567B4010A90000F7402F0D22F801BE51A
:105AFB0067B40216C21E7FFF126ED190000F7403A3
:105B0B00F0C2307F02122EB6D22F302F0C90000F26
:095B1B00E0FD7F0F7E001263B172
:015B2400225E
:10582B008F678D688B69E567700C12586F749F2FAB
:10583B00F58274008019E567B4010C12586F749FE0
:10584B002FF58274008016E567B402091258773E73
:10585B00F583E4F022E567B403091258773EF5832C
:10586B007401F022AD69AF68126EB522AD69AF68F5
:0B587B00126EB5746F2FF582740022CE
:02690B008F6794
:10690D00AF057804EF08800123D8FD4BF568E567E6
:10691D00B40908E568B499030253C7AD68AF6712AF
:02692D006545BE
:01692F002245
:0D6EB500EF75F00AA47C002DFFEC35F0FE17
:016EC20022AD
:04670C008F688D699C
:10671000C3E569648094E4501BE4F56AC3E56964E9
:1067200080F8E56A648098500BC22FAF6812297E0A
:04673000056A80E88E
:016734002242
:0D6EC300C296007F05126875126482D29697
:016ED000229F
:106D5A00126EC3EF20E0F9C296007F06126875C270
:066D6A00B60000D29622E3
:106D7000126EC3EF20E0F9C296007F04126875C25C
:066D8000B60000D29622CD
:046014008E608F61AA
:10601800AE04AF058E638F64C296007F0312687565
:10602800E560FF126875AF61126875E4F562126485
:1060380082E5642562F582E43563F583EFF0056255
:09604800E562C3942040E7D29602
:01605100222C
:085C51008E658F668C678D687B
:105C5900126EC3EF20E0F985656A85666BC296000E
:105C69007F02126875E567FF126875AF681268757B
:105C7900E4F569E56B2569F582E4356AF583E0FFAA
:105C89001268750569E569C3942040E7C2B600004A
:025C9900D296A1
:015C9B0022E6
:0A55E9008E5A8F5B8C5C8D5D8B5E2B
:1055F300C2AF126D5A126EC3EF20E0F9855C60856D
:105603005D61C296007F02126875E55AFF126875E4
:10561300AF5B126875E4F55FAF5EEF3395E0FEC3F1
:10562300E55F9FEE6480F87480985014E561255F10
:10563300F582E43560F583E0FF126875055F80D875
:0B564300C2B60000D296126D70D2AF0C
:01564E002239
:1063B1008E718F728D73C2AF126D5A126EC3EF2040
:1063C100E0F9C296007F02126875E571FF126875E7
:1063D100AF72126875AF73126875C2B60000D296BB
:0663E100126D70D2AF2224
:1060CC00C2AFE4F55BF55CF55DF55EF55FF55AAED8
:1060DC005EAF5FAC5BAD5C1260147420255CF55C4C
:1060EC00E4355BF55B7420255FF55FE4355EF55EAA
:0B60FC00055AE55AC3948940D6D2AF84
:016107002275
:105E0A00C2AF756200756300756400E4F560F56100
:105E1A00F55F126D5AAE63AF64AC60AD61125C514E
:105E2A0074202561F561E43560F56074202564F518
:105E3A0064E43563F563055FE55FC3948940D31273
:045E4A006D70D2AFF6
:015E4E002231
:105713000500050105030507050F051F051E051CEB
:10572300051805100201040E040A03060101040B07
:105733000304040F020304010302040D0200020226
:10574300030004090404030503070100030304071A
:10575300030104060402040C0516051500000615D2
:0E576300062A060C06380633061E0612061726
:104CA5002430F58274003EF583EDFF3395E0FEE593
:104CB500822FF582E5833EF583E0FFEDFB3395E03A
:104CC500FA22AF41126875C293126F1CD293D2AF0C
:104CD500223EF583E0FC74B82FF582741D3EF58302
:104CE500ECF00D221528E528D394002225E02413A5
:104CF500F582E43457F583E49322E4F57CD20EC2C1
:104D050027C21DC21A227FA0126ED1E4F542C21E2F
:104D150022126F1CD2B67801EF0822122C30D2CAAB
:0F4D2500D20ED22722ECFF3395E0FEEF78032267
:10415300200E2F900540E004F577D36480948150BE
:1041630003024213D3E5776480948F400375770F7E
:10417300900029E0FF122C3090002AE0F576124CD3
:10418300FF22301A58302712124CE940030242131F
:10419300C2CAC227D21D85762822301D0A124CE9D5
:1041A300506EC227C21D22AF7A157AEF700BC21A66
:1041B300E57625E0F528D21D22E57B30E0058576FE
:1041C300288008E57675F003A4F528AF7B7801EF26
:1041D30008800103D8FDF57BD227D2CA22D5770800
:1041E300C20EE4F542C21E22057C7440257CF58292
:1041F300E43405F583E0124CF1540FF57A7401931E
:10420300F57B700AD21DE57625E025E0F528D21A64
:014213002288
:1050F200200E12900029E0FF122C3090002AE0F5D9
:1051020078124CFF22301A5130270F124CE9505DB1
:10511200C2CAC227D21D85782822301D0A124CE944
:10512200504BC227C21D22AF7A157AEF7007C21AFE
:10513200C20EF54222E57B30E0058578288008E53D
:105142007875F003A4F528AF7B7801EF088001039E
:10515200D8FDF57BD227D2CA22E543124CF1FA746C
:0D5162000193FBEA540FF57AEBF57BD21AAE
:01516F00221D
:10648200E4F575D297F574C2B6126F1CAF75780138
:10649200EF08800123D8FDF575309703437501128B
:1064A2006F1CD2B60574C3E5746480948840D8AF7B
:0164B2007574
:0164B30022C6
:096F1C000000000000000000224A
:10666100C2B7E4FEC2B6126F1CEF30E704D2B580A8
:1066710002C2B5124D16800123D8FDFF126F1C0E08
:0B668100BE08E1C2B6D2B7D2B6D2B557
:01668C0022EB
:0D001600C2AFEF4227AF27126661D2AF22C2
:0E6ED100C2AFEFF45227AF27126661D2AF2294
:10687500E4FEC2B6126F1CEF30E704D2B58002C247
:10688500B5124D16800123D8FDFF126F1C0EBE08F0
:05689500E1D2B6D2B50E
:01689A0022DB
:096F2500C2AFEF4241124CC72239
:0A6F1200C2AFEFF45241124CC72247
:102C3000EF123A4A2C98012C9F022CA6032CAD04CB
:102C40002CB4052CBB062CC2072CC9082CD0092C8F
:102C5000D70A2CDE0B2CE50C2CEC0D2CF30E2CFAE9
:102C60000F2D01102D08112D0F122D16132D1D14CF
:102C70002D24152D2B162D32172D39182D40192DD9
:102C8000471A2D4E1B2D551C2D571D2D5E1E2D65D3
:102C90001F2D6C2000002D5575CB8E75CAC6227570
:102CA000CB9575CA772275CB9B75CA692275CBA067
:102CB00075CABA2275CBA675CA332275CBAB75CA55
:102CC000632275CBB075CA022275CBB475CAA32234
:102CD00075CBB875CAFA2275CBBC75CAD82275CB2C
:102CE000C075CAA82275CBC475CA362275CBC77504
:102CF000CA862275CBCA75CABC2275CBCD75CAB43B
:102D00002275CBD075CA762275CBD375CA302275A1
:102D1000CBD575CAB22275CBD875CA132275CBDA5A
:102D200075CA522275CBDC75CA7D2275CBDD75CA9A
:102D30006E2275CBE075CA542275CBE275CA1B2290
:102D400075CBE375CAC32275CBE575CA5E2275CB18
:102D5000E675CADA22801C75CBE875CA902275CB5D
:102D6000EA75CAD92275CBEC75CA092275CBED7507
:0A2D7000CA292275CBE875CA41227A
:10002600C3EF648094A15008EF25E025E0F528226F
:04003600E4F52822A3
:02379F008F5A3F
:1037A100900118E0FFE55A7006E545D39F5012E5F8
:1037B1005A64016003023895E546D39F50030238ED
:1037C10095E55A7018C3E5459FF55D74602FF58244
:1037D100E4341EAD82F55E8D5F7F40801BE55AB4F7
:1037E1000119C3E5469FF55D74B02FF582E4341EDF
:1037F100AF82F55E8F5F7F101200167FF47E01129B
:103801006C5B7D207F051266B87D1A7F081266B851
:103811007FC87E00126C5BE4F55BE55BC3955D5090
:1038210061055FE55FAE5E7002055E14F5828E8311
:10383100E0F55C123A4A38720038500A38540B38B5
:103841005A0C38600D38660E386C0F00003878E479
:10385100FD80277D5F7F0780227D5E7F06801C7D46
:103861000A7F0280167D327F0280107D467F0280B2
:103871000A7D0A7F038004AD5CE4FF1266B8055B34
:103881008098E55A70047F408007E55AB401057FAE
:0438910010126ED1D2
:013895002210
:10506F00200E10754406901DB8E06003D20E22E4A6
:10507F00F54222E528D394004003152822C2CA1511
:10508F0044E54414603D14603214601D146015141F
:10509F007049901DB8E0FF7003F54222122C30903A
:1050AF001DB9802F901DBA8015901DBBE0FF7003B6
:1050BF00F54222122C30901DBC8018901DBDE0FFD0
:1050CF00020026901DBEE0FF7003F54222122C3025
:1050DF00901DBFE0FF120026D2CA22E4F542C2CAD9
:0350EF00C20E22CC
:10663300900028E0FF6026200E07124D20752814D5
:1066430022E528D394004003152822202708D2CA24
:0E665300752814D22722C2CA75287DC22722BC
:1065D500200E0C7F1C124D2075286475793C22E530
:1065E50028D394004003152822AF791579D3EF6499
:0E65F500809480400475286422C20EE4F542B2
:016603002274
:10630E00E54214601C14601C14601F14602214609B
:10631E002224057021C2CAC20EC227C21DE4F54452
:10632E002202506F126633D21E22124153D21E2207
:07633E000265D51250F222A6
:10641C00BF010790002A7418F022BF020790002ACF
:10642C007412F022BF030590002A8014BF04079059
:10643C00002A740BF02290002ABF05047409F02284
:04644C00740CF022BA
:024FE900AC0713
:104FEB00C3EC64809480404AEC64809488504320E6
:104FFB002B21E4FD124D2AC333CE33CED8F9124CFC
:10500B00A574102BF58274003AF583EFF00DBD08F3
:10501B00E3801FE4FD124D2AC333CE33CED8F912F1
:10502B004CA574182BF58274003AF583EFF00DBD87
:10503B0008E3202B16E4FDEDFF3395E0FE74102FF3
:10504B00F5827400124CD6BD08ED22302B15E4FD11
:10505B00EDFF3395E0FE74182FF5827400124CD6D9
:03506B00BD08ED90
:01506E00221F
:1053C7007D3F7F091266B87D507F081266B8906FDF
:1053D7004E12542E7D5B7F061266B8906F4F1254A3
:1053E7002E906F50E493FDE4FF1266B8906F51E47E
:1053F7009324BE601414601514601814601B1460A5
:105407001E240570217D0A80067D3280027D467F3D
:105417000280107D0A7F03800A7D287F0380047D38
:10542700467F031266B822E493FDE4FF1266B822B2
:105F56008F5BE55B7005D22DFF8009E55BB4010719
:105F6600D22D7F011259E77D4B7F021266B87D0262
:105F7600E4FF1266B87D32E4FF1266B81253C7E535
:105F86005B70028005E55BB401057F40126ED1228D
:103D1E00A209300501B350307D017F04124ED950F7
:103D2E002320050E30090B9000A4E0FF7C0B7D6074
:103D3E00800F30050F20090C9000A5E0FF7C0B7D55
:103D4E0080125C06A2099205A20A300601B3503019
:103D5E007D027F04124ED9502320060E300A0B909E
:103D6E0000A6E0FF7C0B7DA0800F30060F200A0C12
:103D7E009000A7E0FF7C0B7DC0125C06A20A9206A3
:103D8E00A20B300701B350307D037F04124ED95081
:103D9E002320070E300B0B9000A8E0FF7C0B7DE07C
:103DAE00800F30070F200B0C9000A9E0FF7C0C7DDC
:103DBE0000125C06A20B9207A20D300801B3503020
:103DCE007D047F04124ED9502320080E300D0B9027
:103DDE0000AAE0FF7C0C7D20800F30080F200D0C18
:103DEE009000ABE0FF7C0C7D40125C06A20D9208A9
:013DFE0022A2
:10651500534103900024E0FE543FFF7804088001B6
:1065250023D8FD54F0FFEE30E40343070490002424
:0F653500E030E503430708EF4241C2AF124CC705
:016544002234
:02297E008F6B5D
:10298000302F05756CF48003756C64E56B64017021
:1029900029AF417803EF08800123D8FD3392307FBF
:1029A0001020300B122A9A7F10126F12022A9212F4
:1029B0002AA57F10126F25022A92E56B6402702807
:1029C000AF417802EF08800123D8FD3392307F2099
:1029D00020300A122A9A7F20126F128008122AA52C
:1029E0007F20126F25022A92E56B64037028AF41A5
:1029F0007801EF08800123D8FD3392307F402030EA
:102A00000A122AB07F40126F128008122ABB7F4040
:102A1000126F25022A92E56B6404701EE541339221
:102A2000307F8020300A122AB07F80126F12800817
:102A3000122ABB7F80126F258058E56B64057027D2
:102A4000AF417805EF08800123D8FD3392307F0431
:102A500020300A122AC67F04126F128008122AD16F
:102A60007F04126F25802BE56B6406702CAF4178D4
:102A700004EF08800123D8FD3392307F0820300A0C
:102A8000122AC67F08126F128008122AD17F0812FC
:092A90006F25AF6C7E00126C5B37
:102A990022126F25AF6C7E00126C5B22126F12AF8F
:102AA9006C7E00126C5B22126F25AF6C7E00126C7B
:102AB9005B22126F12AF6C7E00126C5B22126F25C3
:102AC900AF6C7E00126C5B22126F12AF6C7E00122B
:032AD9006C5B2211
:105D7900900024E030E0057F10126F25900024E0A8
:105D890030E1057F20126F25900024E030E2057F85
:105D990040126F25900024E030E3057F80126F25C3
:105DA900900024E030E4057F04126F25900024E080
:095DB90030E5057F08126F252278
:106CC70030030A124D0BC203C211C21E223004093F
:0A6CD700124D0BC204C213C21E22AC
:106545008F708D71E570B4011FE5717003125C9C4D
:10655500E571B401077880E6FF125A8AE571B43215
:106565000E7FF47E01026C5BAD71AF701266B822CE
:1066B800EFFEEDFF1280008E2D8F2E12535275744F
:1066C80032AF741574EFD39400400EE4F573E5739C
:0966D800C3943A50EC057380F5FF
:0166E1002296
:10535200D2A8AFA875A881C214852E82852D83E4B8
:1053620093C4540FFE4306F08E80C284D28500C2DD
:10537200870000D287007580FF7580FEC284C285D7
:1053820000C2870000D287007580FFD2147D407C66
:105392001FE4FE30B40D0EBE32F9ED1D70011CED9E
:1053A2004C70EE7C1F7D40E4FE20B40D0EBE32F93F
:1053B200ED1D70011CED4C70EE8FA8C2A87F0A7E15
:0453C20000126C5B0E
:0153C60022C4
:1066E2007580FDC284C28500C28700000000D28787
:1066F200007580FF7F0A7E00126C5B7F997E091213
:0A67020080008E2D8F2E12535222BC
:10421400D284D285C286A2809217A2819220A282E1
:104224009218A2839221D2862001537D027F01122B
:104234004ED940137D037F01124ED9400A3017072F
:10424400301932D22480377D027F01124ED9500FAB
:1042540030170C302009301904D224802180167DB7
:10426400037F01124ED9501220170330200C30194D
:1042740004D22480091267AF8004C219C224200228
:104284004E7D027F02124ED940127D037F02124EF0
:10429400D94009301806301B2FD225227D027F0217
:1042A400124ED9500E30180B302108301B03D22582
:1042B4002280157D037F02124ED9500F201803303F
:1042C4002109301B03D225220267D7C21BC2252233
:1067AF00753D1E753E60E4FFE53E2FF582E4353DF5
:1067BF00F583E4F00FBF50F0753D1E753E60E4F5B4
:0767CF0045C226C211D219D8
:0167D60022A0
:1067D700753F1E7540B0E4FFE5402FF582E4353F75
:1067E700F583E4F00FBF10F0753F1E7540B0E4F578
:0767F70046C228C213D21BA9
:0167FE002278
:106C0500C284D285C286A2809209A281920AA282FA
:0D6C1500920BA283920DD286D284D28522EA
:10614400E57E2560F582E4357DF5832274FF123AFD
:1061540020E4FBFAF9F8C3023A0D057F7480257E2A
:10616400F57EE4357DF57D22F582E4341DF5832248
:0B617400757F01757D00757E20E42220
:1042D4007D027F07124ED950057F04126F12C22946
:1042E400D223E4F5427FE87E03126C5BC298C2AF2E
:1042F400C2307F03122EB6755E7F755D96755C982D
:10430400755B00785B126150504430983E12000691
:10431400126E28EF14601824F0602624C1600B2468
:10432400F670287F06126F37802112622E801C7F60
:1043340006126F371269E3126515125E0AD22980DC
:104344000A7F06126F37125A3AD2293029B5E47817
:1043540085F6D2307F01122EB67F40120016C22F8E
:1043640012699D7D467F021266B87D1E7F07126624
:10437400B87D147F081266B87D327F031266B8C216
:0D438400307F03122EB67FFF126ED1C223D0
:014391002209
:105A3A00126174F55F7F02126F37E57F2402F56108
:105A4A00AF7F126F37E4F560126144E0FF126F37DF
:105A5A00126144E02561F5610560E560C394804008
:105A6A00E7AF61126F377F03126F37126F3FEF6430
:0F5A7A0015600C12615E055FE55FC3942240B6B4
:015A890022FA
:1069E300126174F55F12673550077F06126F3780A7
:1069F300057F15026F3712615E055FE55FC3942261
:026A030040E36E
:016A0500226E
:10673500E4F560126F3F74D0256012616CEFF005CF
:1067450060E560C3948440EB126E06901E52E0B57E
:086755000705126C76D322C384
:01675D002219
:106C7600E4FF74D22FF582E4341DF583E0FEE57E51
:0A6C86002F126148EEF00FBF7FE807
:016C900022E1
:106E0600E4FFFE74D02E12616CE02FFF0EBE82F3FB
:016E16002259
:10622E00E4F55FF5657564E0756393756204F56179
:10623E00786112615050213098F61200068F60E599
:10624E006064046013AF65056574D02F12616CE550
:08625E0060F0255FF55F80D8B8
:016266002215
:04000600AF99C29854
:01000A0022D3
:086F37003099FDC2998F9922E7
:076F3F003098FDAF99C298E4
:016F46002228
:106D14000C0102030405060708090A0B0C0102030F
:086D24000405060708090A0B2B
:10675E00AF5FEF3395E0FE75F007EF123A3EEE7540
:10676E00F007A42583F583E0227883E6FF126CFB05
:09677E00EF22C295D297D2AF229E
:10689B00C22CC2AF126F477F83126D2C126B141276
:1068AB0067807884E66F600B125E92302B05125F67
:0568BB0096922CA22CB6
:0168C00022B5
:105F96007984E778876660367884E6FF7887F6EF57
:105FA6007013E552C3940A500C7D077F04124ED934
:105FB6005003125E4F7D057F04124ED95010E54105
:105FC60054036005123FB6D322123FB6C322C32242
:103FB600E4F55F900A5012675E700302407A900A39
:103FC600511267656016788166600302407A900A2E
:103FD6005212675E788866600302407AAF5FEF33FD
:103FE60095E0FE900A53126765FF7880E6FEEF6E55
:103FF6006020EF601DB4080BEED394014005EE94EB
:1040060007400FEF6409706CEE64016005EE64070B
:104016007062AF5FEF3395E0FE900A54126765FF5A
:10402600F46006EF788366704BE55FFD3395E0FC40
:10403600900A5575F007ED123A3EEC12676D7884DA
:10404600667031D201D20274BD2DF58274003CF542
:1040560083E0FFC007EDAE047805C333CE33CED878
:10406600F92480F582740E3EAD82FCD007125C0600
:10407600C201C202055FC3E55F64809493500302E8
:024086003FB940
:014088002215
:105E4F007D087F04124ED9500D7883E6FF126CFB4C
:105E5F00EFC39407402CD2307F01122EB67F401231
:105E6F000016C22F12699DD201D202E4FD7F0A12E1
:105E7F004F61C201C2027F50126ED1C2307F011238
:035E8F002EB6220A
:105E9200C2AF126F477FBF126D2C126B147884A6AB
:105EA20007126B147884A607126B147883A6071264
:105EB2006B147888A607126B147881A607126B14EC
:105EC2007880A607126B147882A607126F471267B2
:025ED20080222C
:10588600C2AF126F477F8E1258D57F90126D2C7F54
:10589600A7126D2C126F477FBE126D2CE4FF126D9E
:1058A6002C7884E6FF126D2C7883E6FF126D2C7837
:1058B60088E6FF126D2C7881E6FF126D2C7880E663
:1058C600FF126D2C7882E6FF1258D51267802212DD
:0B58D6006D2CE4FF126D2C126F4722B6
:105A8A008F72E572B401047D63803EE572B402064A
:105A9A007D087F068035E572B403067D317F088074
:105AAA002AE572B404067D617F08801FE572B40599
:105ABA00067D257F088014E572B406067D597F03AA
:0F5ACA008009E572B407077D487F071266B8228E
:026CFB00AE07E2
:106CFD00EE54F0FF780408800103D8FD75F00AA466
:066D0D00FFEE540F2FFF02
:016D1300225D
:105C9C00126777906D1493FF1235A478841267798C
:105CAC00601B7884126779C3940A50077D327F0693
:105CBC001266B87884E6FF126CFB1235A412677773
:105CCC00C3940C50067D0A7F0280047D507F06121F
:0A5CDC0066B87D507F051266B822FD
:105991007FF47E01126C5B7D097F061266B8788107
:1059A1001259D77D0E7F031266B87D357F061266C8
:1059B100B87D097F061266B878881259D77D1E7F97
:1059C100091266B87D1E7F071266B87882E6FF125B
:1059D1006CFB1235A422E6FF126CFB1235A47FF496
:0659E1007E01126C5B2246
:076F4700C2B6C295D29522EB
:106D2C00E4FEC297EF30E002D297C2B6D2B6EFC300
:066D3C0013FF0EBE08EC7F
:016D4200222E
:106B1400E4FFD297FED2B6C2B6A297E433C43333AD
:0F6B2400335480FDEFC313FFED42070EBE08E6AA
:016B3300223F
:1057CE00EF3395E0FE74702FF58274003EF583E0A2
:1057DE00FF22AF5AEF3395E0FEEF222460F582747C
:1057EE00013EAD82FCD22922900520E0F547A3E0D0
:1057FE00F548222450F58274053EAD82FC229000BD
:10580E00BAE0FF7C0E7D2022D222D201E4FF22C21A
:0D581E0001C2227F1922D222D2307F022245
:10281D00E5527008126EFB8F52022918E552B4056D
:10282D00081243928F52022918E552B40B08126C0C
:10283D00918F52022918E552B40A08125CE68F52A4
:10284D00022918E552B40F0812608F8F5202291811
:10285D00E552B414081223368F52022918E552B4EA
:10286D001908126B718F52022918E552B41E081205
:10287D006A4C8F52022918E552B42308126AB28F9E
:10288D0052022918E552B42807126EDF8F52807B51
:10289D00E552B42D071268278F52806FE552B4327E
:1028AD00071262678F528063E552B43E07126B8F39
:1028BD008F528057E552B43C07126DD08F52804B2A
:1028CD00E552B43307126A908F52803FE552B441FE
:1028DD0007126E598F528033E552B44C07126E6950
:1028ED008F528027E552B44407126E798F52801BA8
:1028FD00E552B437071256B48F52800FE552B439F2
:10290D00071254378F528003E4F552E553700612C7
:10291D00000E8F5322E553B40506126F2E8F5322EE
:10292D00E553B40A06126E898F5322E553B40F0690
:10293D00126E988F5322E553B41406123B5A8F53DF
:10294D0022E553B43D06126BAD8F5322E553B43FD0
:10295D00061265758F5322E553B443061267FF8F38
:10296D005322E553B44D06126AD38F5322E4F55327
:01297D002237
:0D6EFB0090052AE0F52BA3E0F52C7F052281
:10439200302414201011C21C7D047F01124ED9500A
:1043A200037F0B227F0A227F0812634550061245C3
:1043B200BE7F0022202408301005C2107F05227D16
:1043C200057F06124ED9501EE53945387018900007
:1043D200B5E0FF7C0D7D80125C0690052EE0F5387D
:1043E200A3E0F53980557D067F06124ED9501EE5B1
:1043F2003C453B70189000B6E0FF7C0D7DA0125C3E
:1044020006900530E0F53BA3E0F53C802E7D077F6A
:1044120005124ED9500D30000AE52C452B7004C20E
:10442200008018300F0AE52C452B7004C20F800B58
:104432007885E6B405057F04125170E55170087560
:0A444200510AD22B12689B7F05225D
:106C9100200F1590053BE0F54E2024037F0522E5EA
:0B6CA1004ED3940050F3D20F7F0A2264
:105CE6007D077F05124ED9500C7D077F05124ED9D0
:105CF600503230002F7D017F01124ED95026D2300E
:105D06007F01122EB67F011200167D027F07124E0A
:105D1600D950057F04126F259000A0E0FF7C0A7D14
:0A5D2600E0125C061257F67F0F2210
:10608F00302437E5484547700C7D087F01124ED903
:10609F0050037F372230030EE53A700A126CC77F28
:1060AF000112001680113026037F14227885E6B482
:0D60BF0005057F031251707F0F227F142210
:1023360090053DE0F54B7F01126ED1126CC77D0210
:102346007F07124ED95009E54B70057F04126F12B4
:102356009000A1E0FF7C0B7D00125C06D22B126878
:102366009BE54570030224607C017D001224DE504B
:10237600037F3E227C017D501224BE50037F3C2207
:102386007C017D581224BE50037F3C227C017D10C7
:102396001224C650081224CE50037F33227C017DBE
:1023A600201224C6500B9000BBE0FF7C0E7D4080BF
:1023B600207C017D281224D6500512580C80127CF0
:1023C600017D301224D650129000B9E0FF7C0E7DBC
:1023D60000125C061267AF7F00227C017D40D22985
:1023E600E4FF1247D3500C7D067F04124ED95003EA
:1023F6007F4C227C017D381224DE50037F44227CF0
:10240600017D18C229E4FF1247D3500C7D057F01D8
:10241600124ED950037F4122E4F55A1257E0780351
:10242600C333CE33CED8F91257E9E4FF1247D3505F
:102436001BAF5A1257CEC0071257E07805C333CEEA
:1024460033CED8F9125801D007125BBB055AC3E543
:102456005A648094A840C47F19221224CE500C7D61
:10246600077F05124ED9504130003E7885E670044C
:102476007F0180087885E6B404077F0212517080D8
:10248600257D037F06124ED9501CE557455670161A
:102496009000AFE0FF7C0C7DC0125C06900532E038
:1024A600F556A3E0F5577F19227D077F05124ED911
:0724B60050052000027F0524
:1024BD0022D229E4FF1247D322D229E4FF1247D3B7
:1024CD00227D077F05124ED922D229E4FF1247D370
:0924DD0022C229E4FF1247D322B8
:106B71003026031267AF7D077F05124ED9500620DC
:0E6B810000037F0522900538E0F54E7F1E22AE
:106A4C00E54E70037F23227D027F07124ED9500939
:106A5C00E54B70057F04126F123024037F0A227FEE
:026A6C001E22E8
:106AB2001257F67D067F01124ED9500C9000ACE0C1
:106AC200FF7C0C7D60125C06900539E0F54E7F2D4F
:016AD20022A1
:0E6EDF007FA0126ED1900539E0F54E7F2D2276
:10682700D22B12689B7D027F07124ED95009E54B88
:1068370070057F04126F12E54E70037F32223024F9
:07684700037F0A227F2D22CE
:10626700301E037F32227D047F06124ED9501FE570
:1062770055455470199000B0E0FF7C0C7DE0125C2E
:1062870006900534E0F554A3E0F5557F3222C2307D
:086297007F01122EB67F0022E8
:106DD00020220CD222E4FF12055BC2227F00227F18
:026DE0003C2253
:106B8F00202218D2227F40120016D201121D7DC280
:0E6B9F00017F40126ED1C2227F19227F3E225A
:106E590020220A12581612379F12581D227F4122EA
:106E690020220A12581612610812581D227F442244
:106E790020220A12581612558012581D227F4422C8
:05000E0000007F052247
:096F2E003025037F0A227F0522B1
:0F6E89009000A2E0FF7C0B7D20125C067F0F22A1
:0F6E98003025093028037F14227F0F227F142218
:103B5A009000A3E0FF7C0B7D40125C06E5467003F3
:103B6A00023C327D017F03124ED950707C017D08E0
:103B7A00C2297F011247D350037F3F227C017D5027
:103B8A00123C3550037F3D227C017D58123C355052
:103B9A00037F3D227C017D40D2297F011247D35009
:103BAA000C7D067F04124ED950037F4D227C017D85
:103BBA0028D2297F011247D3500912580C125C06E9
:103BCA007F00227C017D18C2297F011247D3500C45
:103BDA007D057F02124ED950037F43227D027F0367
:103BEA00124ED95043E4F55AAF5A1257E27803C33A
:103BFA0033CE33CED8F91257E97F011247D3501D7D
:103C0A00AF5A1257CEC007AF5A1257E27805C333DC
:103C1A00CE33CED8F9125801D007125BBB055AC36E
:0A3C2A00E55A648094A840C07F00B2
:093C340022D2297F011247D3229C
:106BAD00202218D222C2307F01122EB67F01126E22
:0E6BBD00D17F0112055BC2227F00227F3D22A4
:1065750020222A125824122EB67FF47E01126C5B5B
:106585007F10120016D202121B7CC2027F10126EFF
:10659500D1C2307F02122EB6C2227F00227F3F2257
:1067FF00202222125824122EB67FF47E01126C5BD7
:10680F00D2027F0112379FC202C2307F02122EB610
:08681F00C2227F00227F432208
:106AD30020221B125824122EB6D2027F0112610803
:106AE300C202C2307F02122EB6C2227F00227F4D25
:016AF3002280
:1054A700AF5AEF3395E0FE22900520E0F547A3E0E1
:1054B700F54822900522E0F549A3E0F54A22246049
:1054C700F58274013EAD82FCD2292274702FF582D9
:1054D70074003EF583E0FF22C202C2227F19222414
:1054E70050F58274053EAD82FC22900536E0F53218
:1054F700A3E0F53322055AC3E55A648094A822D263
:0D55070022C2307F0122D222C2307F022258
:10325100E5527006126A6E8F5222E552B4050612CB
:1032610036A38F5222E552B40B0612684E8F5222BA
:10327100E552B40A0612444C8F5222E552B40F06AD
:10328100126DE28F5222E552B411061259398F5252
:1032910022E552B412061251EA8F5222E552B414B9
:1032A10006120A548F5222E552B419061266048F8F
:1032B1005222E552B41E061265A58F5222E552B480
:1032C1002306125F158F5222E552B42806126EEDC5
:1032D1008F5222E552B42D0612617F8F5222E552A0
:1032E100B4320612629F8F5222E552B43C06126D2F
:1032F100F48F5222E552B43D06126CAC8F5222E596
:1033010052B43E061269308F5222E552B43F061282
:103311006E178F5222E552B44106126B348F52223E
:10332100E552B44306126A068F5222E552B44C06A6
:10333100126CE18F5222E552B44D06126A298F5266
:1033410022E552B437061256B48F5222E552B439EF
:10335100061254378F5222E552B4380612668D8F09
:103361005222E552B43306126A908F5222E552B4CA
:0C3371004406126D438F5222E4F55222F4
:106A6E0090052AE0F52BA3E0F52C7D067F02124E51
:106A7E00D9500C90052CE0F529A3E0F52AD21F7F02
:026A8E000522DF
:1036A300302414201011C21C7D047F01124ED95006
:1036B300037F0B227F0A22302514201211D21C7D96
:1036C300047F02124ED950037F0B227F0A227F0808
:1036D30012634550061245BE7F0022202408301095
:1036E30005C2107F0522202508301205C2127F056E
:1036F300227D057F06124ED9501EE53945387018D4
:103703009000B5E0FF7C0D7D80125C0690052EE0F5
:10371300F538A3E0F53980757D067F06124ED95042
:103723001EE53C453B70189000B6E0FF7C0D7DA084
:10373300125C06900530E0F53BA3E0F53C804E7D3E
:10374300077F05124ED9500D30000AE52C452B702A
:1037530004C200800B300F08E52C452B7002C20F0A
:103763007D067F02124ED95019301F16E52A4529CE
:103773007010C21F9000BCE0FF7C0E7D60125C06DF
:10378300800B7885E6B405057F04125170E551700E
:0C3793000875510AD22B12689B7F05229A
:10684E00200F2190053BE0F54E202406201C037FEF
:10685E000522202506301C037F0522E54ED3940029
:07686E0050E7D20F7F0A2260
:10444C007D077F05124ED950127D077F05124ED97C
:10445C0040030244FD2000030244FD201C3FD230E7
:10446C007F03122EB67F0F126ED190000FE0B402B4
:10447C00047F05800990000FE0B403057F01120052
:10448C00161254AF7D027F07124ED950057F0412CD
:10449C006F259000A0E0FF7C0A7DE0804E301C511F
:1044AC0090000FE0FF64026005EF640370437F0F20
:1044BC00126ED17F05126345400BD2307F01122E54
:1044CC00B67F028009D2307F03122EB67F0A12000B
:1044DC00167D027F07124ED950057F04126F2512EC
:1044EC0054BA9000A2E0FF7C0B7D20125C067F0F7B
:0A44FC00221254AF1254BA7F0F22AF
:106DE200201C063024037F1122301C053025027F2F
:026DF20012226B
:10593900302452E5484547700C7D087F01124ED945
:1059490050037F3722300329E53A70257FA0126E74
:10595900D190000FE0B401047F01800990000FE0AD
:10596900B402057F05120016E4F542C21EC2038087
:10597900113026037F14227885E6B405057F0312CA
:0859890051707F11227F1422EE
:1051EA00301C1030240D20100A7F0A126ED1C21C06
:1051FA007F0A22301C4C3025492012463003031204
:10520A006CC7E54A4549700C7D087F02124ED95099
:10521A00037F3822300417E53A70137FA0126ED14B
:10522A007F02120016E4F542C21EC2048011302821
:10523A00037F14227885E6B405057F031251707F37
:10524A001222201C1230250F20120CD21CC2307FD1
:0A525A0002122EB67F0A227F1422F2
:100A540090053DE0F54B7F0F126ED1201C0C9000E9
:100A6400A1E0FF7C0B7D00125C06301C0C9000A3FF
:100A7400E0FF7C0B7D40125C06E542B403037F1467
:100A840022126CC7E4F5427D027F07124ED9500949
:100A9400E54B70057F04126F12D22B12689B301C39
:100AA40003020B97E5457003020B977C017D00124E
:100AB4000D1450037F3E227C017D50120CE4500340
:100AC4007F3C227C017D58120CE450037F3C227C45
:100AD400017D10120CEC5008120CFC50037F3322E1
:100AE4007C017D20120CEC5003020BFE7C017D285E
:100AF400120D04500C9000BAE0FF7C0E7D20020C15
:100B0400077C017D30120D04500C9000B9E0FF7C8D
:100B14000E7D00020C077C017D40D229E4FF1247C0
:100B2400D3500C7D067F04124ED950037F4C227C97
:100B3400017D38120D1450037F44227C017D18C2BC
:100B440029E4FF1247D3500C7D057F01124ED95082
:100B5400037F4122E4F55A1254A7EF7803C333CE3E
:100B640033CED8F91254C5E4FF1247D3501D1254A2
:100B7400A71254D2C0071254A7EF7805C333CE335B
:100B8400CED8F91254E6D007125BBB1254FC40C70E
:100B94007F1922201C03020C8AE5467003020C8A8A
:100BA4007D017F03124ED94003020C427C017D0873
:100BB400C2297F011247D3500F7F50120016D23042
:100BC4007F02122EB67F3F227C017D50120CF4501E
:100BD400037F3D227C017D58120CF450037F3D229B
:100BE4007C017D10120D0C5008120CFC50037F3355
:100BF400227C017D20120D0C50129000BBE0FF7C82
:100C04000E7D40125C061267AF7F00227C017D409E
:100C1400D2297F011247D3500C7D067F04124ED98E
:100C240050037F4D227C017D18C2297F011247D3D6
:100C3400500C7D057F02124ED950037F43227D0262
:100C44007F03124ED9503CE4F55A1254A7EF7803AF
:100C5400C333CE33CED8F91254C57F011247D350D3
:100C64001D1254A71254D2C0071254A7EF7805C31B
:100C740033CE33CED8F91254E6D007125BBB1254EC
:100C8400FC40C77F1922120D1C5008120D1C504144
:100C940030003E7885E670047F0180087885E6B4EC
:100CA40004077F0212517080257D037F06124ED9FE
:100CB400501CE557455670169000AFE0FF7C0C7D44
:100CC400C0125C06900532E0F556A3E0F5577F1993
:0F0CD400227D077F05124ED950052000027F05B3
:100CE30022D229E4FF1247D322D229E4FF1247D3A9
:100CF30022D2297F011247D3227D077F05124ED9C5
:100D030022D229E4FF1247D322D2297F011247D3EB
:100D130022C229E4FF1247D3227D077F05124ED951
:010D230022AD
:10660400C219C2307F02122EB63026051267AF803F
:10661400063028031267D77D077F05124ED950062E
:0F6624002000037F0522900538E0F54E7F1E22EF
:1065A500E54E70037F23227D027F07124ED95009E5
:1065B500E54B70057F04126F123024062010037F0F
:1065C5000A22302508201205D21C7F0A227F1E22AE
:105F1500201C051254AF80031254BA7D067F01126E
:105F25004ED95024E5427020201C0B9000ACE0FFB8
:105F35007C0C7D60800C301C0C9000ADE0FF7C0C6F
:105F45007D80125C067F2822900539E0F54E7F2D75
:015F55002229
:0E6EED007FA0126ED1900539E0F54E7F2D2268
:10617F00D22B12689B7D027F07124ED95009E54B37
:10618F0070057F04126F12E54E601D30240620103B
:10619F00037F0A2290000FE064016009302506207A
:0B61AF0012037F05227F2D227F322289
:10629F00301E037F32227D047F06124ED9501FE538
:1062AF0055455470199000B0E0FF7C0C7DE0125CF6
:1062BF0006900534E0F554A3E0F5557F3222C23045
:0862CF007F01122EB67F0022B0
:106DF40020220CD222E4FF12055BC2227F00227FF4
:026E04003C222E
:1069300020221FC2307F02122EB6D2227F401200C8
:1069400016D201121D7DC2017F40126ED1C2227F7C
:0569500019227F3E2228
:106E170020220BD222D202121B7C1254DF227F3F88
:016E27002248
:106CAC00202215125506122EB67F40126ED17F018E
:0B6CBC0012055BC2227F00227F3D22F8
:106B340020221912550D122EB67F10126ED1D201D9
:0F6B4400E4FF12379FC201C2227F19227F412234
:106A060020221D125506122EB67F40126ED1D230AC
:106A16007F02122EB6D2027F0112379F1254DF2256
:036A26007F432289
:106CE10020221412550D122EB6D201E4FF126108B2
:0A6CF100C201C2227F19227F412256
:106A290020221D125506122EB67F40126ED1D23089
:106A39007F02122EB6D2027F011261081254DF22A0
:036A49007F432266
:106D430020221112550D122EB6D202E4FF125580E5
:076D53001254DF227F4422ED
:1056B400D2107D027F07124ED950057F04126F125B
:1056C40090000FE0FF64016004EFB4030E7F011249
:1056D4006ED17F401257037F01801390000FE0B416
:1056E400020F7F05126ED17F501257037F03126F92
:1056F400127F50126ED13015031254F17F392212E9
:0F5704000016C22F12699DE4FD7F07124F61222C
:1054370030241130150BE53345327005C23112693E
:10544700557F3922E47885F6C21090000FE0FF649B
:10545700016005EF64037010D2307F01122EB67F12
:10546700401254957F01801B90000FE06402701674
:10547700D2307F03122EB67F05126ED17F501254A1
:10548700957F03122EB67F50126ED17F0022120035
:1054970016C22F12699DE4FD7F08124F61C23022A8
:10668D00D2127F0A126ED17F40120016D22F1269DC
:10669D009DE4FD7F07124F617F03126F127F501231
:0B66AD006ED13015031254F17F002263
:106A900030000B9000B8E0FF7C0D7DE0800C200002
:106AA0000E9000B7E0FF7C0D7DC0125C06B2007F47
:026AB0001922A9
:106108008F5AE55A24FF922F12699DE55A70127F23
:1061180040120016D201E4FD7F09124F61C20180CE
:1061280015E55AB401107F10120016D202E4FD7F63
:0C61380009124F61C2027F50126ED1228A
:104DC100C201C202D20C7F50126ED17F8012001636
:104DD10075420390000FE0B401163024627F011286
:104DE1000016302407E542D3940050F67F01803548
:104DF10090000FE0FF64026005EF6403704130240E
:104E0100297F02126ED1D2307F03122EB67F051296
:104E11000016302407E542D3940050F6C2307F02D9
:104E2100122EB67F05126ED180153025127F021227
:104E3100001630250AE542D3940040033024F3E5FF
:0D4E41004270907FA0126ED1C20CC21E22E2
:03000000026C226D
:106C2200758E0078FEE4F6D8FD9000007FFF7E1F8F
:0D6C3200E4F0A3DFFCDEFA758188024C154A
:10398400C2D530F707B2D563F0FF05F030E70CB2CB
:10399400D5F4048463F0FF05F080018430D502F48B
:0239A4000422FB
:1039A600EF8DF0A4A8F0CF8CF0A428CE8DF0A42E35
:0239B600FE22EF
:1039B800BC000BBE0029EF8DF084FFADF022E4CCF3
:1039C800F875F008EF2FFFEE33FEEC33FCEE9DECBC
:1039D800984005FCEE9DFE0FD5F0E9E4CEFD22ED02
:1039E800F8F5F0EE8420D21CFEADF075F008EF2F4C
:1039F800FFED33FD4007985006D5F0F222C398FD3D
:053A08000FD5F0EA22D9
:103A0D00EB9FF5F0EA9E42F0E99D42F0E89C45F00F
:013A1D002286
:103A1E007401FF3395E0FEFDFC080808E6CF2FF693
:103A2E0018E6CE3EF618E6CD3DF618E6CC3CF6226C
:0C3A3E00A42582F582E5F03583F5832293
:103A4A00D083D082F8E4937012740193700DA3A30B
:103A5A0093F8740193F5828883E47374029368601F
:063A6A00EFA3A3A380DF1F
:106E2800EFC39461400AEF947B5005EF24E0FF2202
:016E38002237
:00000001FF
